 systemclssearch_agent

 Timestamp is 51a78bdd (reproducible build file hash)

 Preferred load address is 0000000180000000

 Start         Length     Name                   Class
 0001:00000000 00003850H .text$mn                CODE
 0001:00003850 00000036H .text$mn$00             CODE
 0001:00003886 00000092H .text$x                 CODE
 0002:00000000 000001c8H .idata$5                DATA
 0002:000001c8 00000038H .00cfg                  DATA
 0002:00000200 00000008H .CRT$XCA                DATA
 0002:00000208 00000008H .CRT$XCZ                DATA
 0002:00000210 00000008H .CRT$XIA                DATA
 0002:00000218 00000008H .CRT$XIC                DATA
 0002:00000220 00000008H .CRT$XIZ                DATA
 0002:00000228 00000008H .CRT$XLA                DATA
 0002:00000230 00000008H .CRT$XLZ                DATA
 0002:00000238 00000008H .CRT$XPA                DATA
 0002:00000240 00000008H .CRT$XPZ                DATA
 0002:00000248 00000008H .CRT$XTA                DATA
 0002:00000250 00000010H .CRT$XTZ                DATA
 0002:00000258 00000000H .gehcont$y              DATA
 0002:00000258 00000000H .gfids$y                DATA
 0002:00000260 00002220H .rdata                  DATA
 0002:00002480 00000000H .rdata$CastGuardVftablesA DATA
 0002:00002480 00000000H .rdata$CastGuardVftablesC DATA
 0002:00002480 00000028H .rdata$T                DATA
 0002:000024a8 000000a8H .rdata$voltmd           DATA
 0002:00002550 00000328H .rdata$zzzdbg           DATA
 0002:00002878 00000008H .rtc$IAA                DATA
 0002:00002880 00000008H .rtc$IZZ                DATA
 0002:00002888 00000008H .rtc$TAA                DATA
 0002:00002890 00000008H .rtc$TZZ                DATA
 0002:00002898 00000004H .tls                    DATA
 0002:0000289c 00000004H .tls$                   DATA
 0002:000028a0 00000008H .tls$ZZZ                DATA
 0002:000028a8 00000388H .xdata                  DATA
 0002:00002c30 00000370H .edata                  DATA
 0002:00002fa0 0000008cH .idata$2                DATA
 0002:0000302c 00000014H .idata$3                DATA
 0002:00003040 000001c8H .idata$4                DATA
 0002:00003208 00000486H .idata$6                DATA
 0003:00000000 00000080H .data                   DATA
 0003:00000080 0001c9a8H .bss                    DATA
 0004:00000000 000003f0H .pdata                  DATA

  Address         Publics by Value              Rva+Base               Lib:Object

 0000:00000000       __AbsoluteZero             0000000000000000     <absolute>
 0000:00000000       ___safe_se_handler_count   0000000000000000     <absolute>
 0000:00000000       ___safe_se_handler_table   0000000000000000     <absolute>
 0000:00000000       __arm64x_extra_rfe_table   0000000000000000     <absolute>
 0000:00000000       __arm64x_extra_rfe_table_size 0000000000000000     <absolute>
 0000:00000000       __arm64x_native_entrypoint 0000000000000000     <absolute>
 0000:00000000       __arm64x_redirection_metadata 0000000000000000     <absolute>
 0000:00000000       __arm64x_redirection_metadata_count 0000000000000000     <absolute>
 0000:00000000       __dynamic_value_reloc_table 0000000000000000     <absolute>
 0000:00000000       __enclave_config           0000000000000000     <absolute>
 0000:00000000       __guard_check_icall_a64n_fptr 0000000000000000     <absolute>
 0000:00000000       __guard_eh_cont_count      0000000000000000     <absolute>
 0000:00000000       __guard_eh_cont_table      0000000000000000     <absolute>
 0000:00000000       __guard_fids_count         0000000000000000     <absolute>
 0000:00000000       __guard_fids_table         0000000000000000     <absolute>
 0000:00000000       __guard_iat_count          0000000000000000     <absolute>
 0000:00000000       __guard_iat_table          0000000000000000     <absolute>
 0000:00000000       __guard_longjmp_count      0000000000000000     <absolute>
 0000:00000000       __guard_longjmp_table      0000000000000000     <absolute>
 0000:00000000       __hybrid_auxiliary_iat     0000000000000000     <absolute>
 0000:00000000       __hybrid_auxiliary_iat_copy 0000000000000000     <absolute>
 0000:00000000       __hybrid_code_map          0000000000000000     <absolute>
 0000:00000000       __hybrid_code_map_count    0000000000000000     <absolute>
 0000:00000000       __x64_code_ranges_to_entry_points 0000000000000000     <absolute>
 0000:00000000       __x64_code_ranges_to_entry_points_count 0000000000000000     <absolute>
 0000:00000100       __guard_flags              0000000000000100     <absolute>
 0000:00000000       __ImageBase                0000000180000000     <linker-defined>
 0001:00000000       ?NewObject@JNIEnv_@@QEAAPEAV_jobject@@PEAV_jclass@@PEAU_jmethodID@@ZZ 0000000180001000 f i libsystemclssearch_agent.obj
 0001:00000028       ?SetEventNotificationMode@_jvmtiEnv@@QEAA?AW4jvmtiError@@W4jvmtiEventMode@@W4jvmtiEvent@@PEAV_jobject@@ZZ 0000000180001028 f i libsystemclssearch_agent.obj
 0001:00000034       ?TranslateError@@YAPEBDW4jvmtiError@@@Z 0000000180001034 f   libsystemclssearch_agent.obj
 0001:000002ec       ?nsk_jni_check_exception@@YAHPEAUJNIEnv_@@QEBDH@Z 00000001800012ec f   libsystemclssearch_agent.obj
 0001:00000430       ?nsk_jni_lverify@@YAHHPEAUJNIEnv_@@HQEBDH1ZZ 0000000180001430 f   libsystemclssearch_agent.obj
 0001:000004d0       Agent_Initialize           00000001800014d0 f   libsystemclssearch_agent.obj
 0001:000008d8       Agent_OnAttach             00000001800018d8 f   libsystemclssearch_agent.obj
 0001:000008d8       Agent_OnLoad               00000001800018d8 f   libsystemclssearch_agent.obj
 0001:000008e0       Java_nsk_jvmti_unit_FollowReferences_FollowRefObjects_addRefToVerify 00000001800018e0 f   libsystemclssearch_agent.obj
 0001:00000ab8       Java_nsk_jvmti_unit_FollowReferences_FollowRefObjects_getTag 0000000180001ab8 f   libsystemclssearch_agent.obj
 0001:00000b78       Java_nsk_jvmti_unit_FollowReferences_FollowRefObjects_resetRefsToVerify 0000000180001b78 f   libsystemclssearch_agent.obj
 0001:00000b80       Java_nsk_jvmti_unit_FollowReferences_FollowRefObjects_resetTags 0000000180001b80 f   libsystemclssearch_agent.obj
 0001:00000bc4       Java_nsk_jvmti_unit_FollowReferences_FollowRefObjects_setTag 0000000180001bc4 f   libsystemclssearch_agent.obj
 0001:00000e1c       Java_nsk_share_jvmti_ArgumentHandler_getAgentOptionsString 0000000180001e1c f   libsystemclssearch_agent.obj
 0001:00000ecc       Java_nsk_share_jvmti_DebugeeClass_checkStatus 0000000180001ecc f   libsystemclssearch_agent.obj
 0001:00000f54       Java_nsk_share_jvmti_DebugeeClass_resetAgentData 0000000180001f54 f   libsystemclssearch_agent.obj
 0001:00000fb4       Java_nsk_share_jvmti_RedefineAgent_agentStatus 0000000180001fb4 f   libsystemclssearch_agent.obj
 0001:00000fc0       Java_nsk_share_jvmti_RedefineAgent_isRedefined 0000000180001fc0 f   libsystemclssearch_agent.obj
 0001:00000fcc       Java_nsk_share_jvmti_RedefineAgent_redefineAttempted 0000000180001fcc f   libsystemclssearch_agent.obj
 0001:00000fd8       MA_checkStatus             0000000180001fd8 f   libsystemclssearch_agent.obj
 0001:0000107c       __local_stdio_printf_options 000000018000207c f i libsystemclssearch_agent.obj
 0001:00001348       callbackVMDeath            0000000180002348 f   libsystemclssearch_agent.obj
 0001:000014ac       callbackVMInit             00000001800024ac f   libsystemclssearch_agent.obj
 0001:000017f8       exitOnError                00000001800027f8 f   libsystemclssearch_agent.obj
 0001:000018ac       fprintf                    00000001800028ac f i libsystemclssearch_agent.obj
 0001:000018f0       nsk_complain               00000001800028f0 f   libsystemclssearch_agent.obj
 0001:0000191c       nsk_jvmti_createJVMTIEnv   000000018000291c f   libsystemclssearch_agent.obj
 0001:00001a4c       nsk_jvmti_enableEvents     0000000180002a4c f   libsystemclssearch_agent.obj
 0001:00001b20       nsk_jvmti_findOptionStringValue 0000000180002b20 f   libsystemclssearch_agent.obj
 0001:00001b90       nsk_jvmti_findOptionValue  0000000180002b90 f   libsystemclssearch_agent.obj
 0001:00001c08       nsk_jvmti_lverify          0000000180002c08 f   libsystemclssearch_agent.obj
 0001:00001cf8       nsk_jvmti_parseOptions     0000000180002cf8 f   libsystemclssearch_agent.obj
 0001:00001f48       nsk_jvmti_resetAgentData   0000000180002f48 f   libsystemclssearch_agent.obj
 0001:00001fc8       nsk_jvmti_setFailStatus    0000000180002fc8 f   libsystemclssearch_agent.obj
 0001:00002004       nsk_lcomplain              0000000180003004 f   libsystemclssearch_agent.obj
 0001:00002024       nsk_ldisplay               0000000180003024 f   libsystemclssearch_agent.obj
 0001:00002044       nsk_ltrace                 0000000180003044 f   libsystemclssearch_agent.obj
 0001:00002064       nsk_lvcomplain             0000000180003064 f   libsystemclssearch_agent.obj
 0001:0000221c       nsk_lvdisplay              000000018000321c f   libsystemclssearch_agent.obj
 0001:00002268       nsk_lverify                0000000180003268 f   libsystemclssearch_agent.obj
 0001:000022c4       nsk_lvtrace                00000001800032c4 f   libsystemclssearch_agent.obj
 0001:00002324       nsk_printf                 0000000180003324 f   libsystemclssearch_agent.obj
 0001:0000234c       nsk_vprintf                000000018000334c f   libsystemclssearch_agent.obj
 0001:00002400       printf                     0000000180003400 f i libsystemclssearch_agent.obj
 0001:00002928       __raise_securityfailure    0000000180003928 f   MSVCRT:gs_report.obj
 0001:0000295c       __report_gsfailure         000000018000395c f   MSVCRT:gs_report.obj
 0001:00002b9c       __GSHandlerCheck           0000000180003b9c f   MSVCRT:gshandler.obj
 0001:00002bbc       __GSHandlerCheckCommon     0000000180003bbc f   MSVCRT:gshandler.obj
 0001:00002c30       __security_check_cookie    0000000180003c30 f   MSVCRT:amdsecgs.obj
 0001:00002f70       _DllMainCRTStartup         0000000180003f70 f   MSVCRT:dll_dllmain.obj
 0001:00002fb0       __scrt_acquire_startup_lock 0000000180003fb0 f   MSVCRT:utility.obj
 0001:00002fec       __scrt_dllmain_after_initialize_c 0000000180003fec f   MSVCRT:utility.obj
 0001:00003020       __scrt_dllmain_before_initialize_c 0000000180004020 f   MSVCRT:utility.obj
 0001:00003038       __scrt_dllmain_crt_thread_attach 0000000180004038 f   MSVCRT:utility.obj
 0001:00003060       __scrt_dllmain_crt_thread_detach 0000000180004060 f   MSVCRT:utility.obj
 0001:00003078       __scrt_dllmain_exception_filter 0000000180004078 f   MSVCRT:utility.obj
 0001:000030d8       __scrt_dllmain_uninitialize_c 00000001800040d8 f   MSVCRT:utility.obj
 0001:00003108       __scrt_dllmain_uninitialize_critical 0000000180004108 f   MSVCRT:utility.obj
 0001:0000311c       __scrt_initialize_crt      000000018000411c f   MSVCRT:utility.obj
 0001:00003168       __scrt_initialize_onexit_tables 0000000180004168 f   MSVCRT:utility.obj
 0001:000031f4       __scrt_is_nonwritable_in_current_image 00000001800041f4 f   MSVCRT:utility.obj
 0001:0000328c       __scrt_release_startup_lock 000000018000428c f   MSVCRT:utility.obj
 0001:000032b0       __scrt_uninitialize_crt    00000001800042b0 f   MSVCRT:utility.obj
 0001:000032dc       _onexit                    00000001800042dc f   MSVCRT:utility.obj
 0001:00003318       atexit                     0000000180004318 f   MSVCRT:utility.obj
 0001:00003330       __crt_debugger_hook        0000000180004330 f   MSVCRT:utility_desktop.obj
 0001:00003338       __scrt_fastfail            0000000180004338 f   MSVCRT:utility_desktop.obj
 0001:00003484       _guard_check_icall_nop     0000000180004484 f i MSVCRT:guard_support.obj
 0001:00003488       __security_init_cookie     0000000180004488 f   MSVCRT:gs_support.obj
 0001:00003534       DllMain                    0000000180004534 f   MSVCRT:dll_dllmain_stub.obj
 0001:00003558       ?__scrt_initialize_type_info@@YAXXZ 0000000180004558 f   MSVCRT:tncleanup.obj
 0001:00003568       ?__scrt_uninitialize_type_info@@YAXXZ 0000000180004568 f   MSVCRT:tncleanup.obj
 0001:00003574       __local_stdio_scanf_options 0000000180004574 f i MSVCRT:default_local_stdio_options.obj
 0001:0000357c       __scrt_initialize_default_local_stdio_options 000000018000457c f   MSVCRT:default_local_stdio_options.obj
 0001:00003598       __scrt_get_dyn_tls_init_callback 0000000180004598 f   MSVCRT:dyn_tls_init.obj
 0001:000035a0       _RTC_Initialize            00000001800045a0 f   MSVCRT:initsect.obj
 0001:000035dc       _RTC_Terminate             00000001800045dc f   MSVCRT:initsect.obj
 0001:00003618       __isa_available_init       0000000180004618 f   MSVCRT:cpu_disp.obj
 0001:000037c4       _get_startup_argv_mode     00000001800047c4 f   MSVCRT:argv_mode.obj
 0001:000037cc       __scrt_is_ucrt_dll_in_use  00000001800047cc f   MSVCRT:ucrt_detection.obj
 0001:000037e0       memcpy                     00000001800047e0 f   vcruntime:VCRUNTIME140.dll
 0001:000037e6       memset                     00000001800047e6 f   vcruntime:VCRUNTIME140.dll
 0001:000037ec       strchr                     00000001800047ec f   vcruntime:VCRUNTIME140.dll
 0001:000037f2       __C_specific_handler       00000001800047f2 f   vcruntime:VCRUNTIME140.dll
 0001:000037f8       __std_type_info_destroy_list 00000001800047f8 f   vcruntime:VCRUNTIME140.dll
 0001:000037fe       strcmp                     00000001800047fe f   ucrt:api-ms-win-crt-string-l1-1-0.dll
 0001:00003804       strlen                     0000000180004804 f   ucrt:api-ms-win-crt-string-l1-1-0.dll
 0001:0000380a       _initterm                  000000018000480a f   ucrt:api-ms-win-crt-runtime-l1-1-0.dll
 0001:00003810       _initterm_e                0000000180004810 f   ucrt:api-ms-win-crt-runtime-l1-1-0.dll
 0001:00003816       _seh_filter_dll            0000000180004816 f   ucrt:api-ms-win-crt-runtime-l1-1-0.dll
 0001:0000381c       _configure_narrow_argv     000000018000481c f   ucrt:api-ms-win-crt-runtime-l1-1-0.dll
 0001:00003822       _initialize_narrow_environment 0000000180004822 f   ucrt:api-ms-win-crt-runtime-l1-1-0.dll
 0001:00003828       _initialize_onexit_table   0000000180004828 f   ucrt:api-ms-win-crt-runtime-l1-1-0.dll
 0001:0000382e       _register_onexit_function  000000018000482e f   ucrt:api-ms-win-crt-runtime-l1-1-0.dll
 0001:00003834       _execute_onexit_table      0000000180004834 f   ucrt:api-ms-win-crt-runtime-l1-1-0.dll
 0001:0000383a       _crt_atexit                000000018000483a f   ucrt:api-ms-win-crt-runtime-l1-1-0.dll
 0001:00003840       _cexit                     0000000180004840 f   ucrt:api-ms-win-crt-runtime-l1-1-0.dll
 0001:00003848       __acrt_initialize          0000000180004848 f   MSVCRT:ucrt_stubs.obj
 0001:00003848       __acrt_thread_attach       0000000180004848 f   MSVCRT:ucrt_stubs.obj
 0001:00003848       __acrt_thread_detach       0000000180004848 f   MSVCRT:ucrt_stubs.obj
 0001:00003848       __acrt_uninitialize        0000000180004848 f   MSVCRT:ucrt_stubs.obj
 0001:00003848       __acrt_uninitialize_critical 0000000180004848 f   MSVCRT:ucrt_stubs.obj
 0001:00003848       __scrt_stub_for_acrt_initialize 0000000180004848 f   MSVCRT:ucrt_stubs.obj
 0001:00003848       __scrt_stub_for_acrt_thread_attach 0000000180004848 f   MSVCRT:ucrt_stubs.obj
 0001:00003848       __scrt_stub_for_acrt_thread_detach 0000000180004848 f   MSVCRT:ucrt_stubs.obj
 0001:00003848       __scrt_stub_for_acrt_uninitialize 0000000180004848 f   MSVCRT:ucrt_stubs.obj
 0001:00003848       __scrt_stub_for_acrt_uninitialize_critical 0000000180004848 f   MSVCRT:ucrt_stubs.obj
 0001:00003848       __vcrt_initialize          0000000180004848 f   MSVCRT:ucrt_stubs.obj
 0001:00003848       __vcrt_thread_attach       0000000180004848 f   MSVCRT:ucrt_stubs.obj
 0001:00003848       __vcrt_thread_detach       0000000180004848 f   MSVCRT:ucrt_stubs.obj
 0001:00003848       __vcrt_uninitialize        0000000180004848 f   MSVCRT:ucrt_stubs.obj
 0001:00003848       __vcrt_uninitialize_critical 0000000180004848 f   MSVCRT:ucrt_stubs.obj
 0001:0000384c       __scrt_stub_for_is_c_termination_complete 000000018000484c f   MSVCRT:ucrt_stubs.obj
 0001:0000384c       _is_c_termination_complete 000000018000484c f   MSVCRT:ucrt_stubs.obj
 0001:00003860       _guard_dispatch_icall_nop  0000000180004860 f   MSVCRT:guard_dispatch.obj
 0001:00003880       _guard_xfg_dispatch_icall_nop 0000000180004880 f   MSVCRT:guard_xfg_dispatch.obj
 0002:00000000       __imp_RtlCaptureContext    0000000180005000     kernel32:KERNEL32.dll
 0002:00000008       __imp_RtlLookupFunctionEntry 0000000180005008     kernel32:KERNEL32.dll
 0002:00000010       __imp_RtlVirtualUnwind     0000000180005010     kernel32:KERNEL32.dll
 0002:00000018       __imp_UnhandledExceptionFilter 0000000180005018     kernel32:KERNEL32.dll
 0002:00000020       __imp_SetUnhandledExceptionFilter 0000000180005020     kernel32:KERNEL32.dll
 0002:00000028       __imp_GetCurrentProcess    0000000180005028     kernel32:KERNEL32.dll
 0002:00000030       __imp_TerminateProcess     0000000180005030     kernel32:KERNEL32.dll
 0002:00000038       __imp_IsProcessorFeaturePresent 0000000180005038     kernel32:KERNEL32.dll
 0002:00000040       __imp_CloseHandle          0000000180005040     kernel32:KERNEL32.dll
 0002:00000048       __imp_InitializeCriticalSectionAndSpinCount 0000000180005048     kernel32:KERNEL32.dll
 0002:00000050       __imp_DeleteCriticalSection 0000000180005050     kernel32:KERNEL32.dll
 0002:00000058       __imp_CreateEventW         0000000180005058     kernel32:KERNEL32.dll
 0002:00000060       __imp_GetModuleHandleW     0000000180005060     kernel32:KERNEL32.dll
 0002:00000068       __imp_GetProcAddress       0000000180005068     kernel32:KERNEL32.dll
 0002:00000070       __imp_IsDebuggerPresent    0000000180005070     kernel32:KERNEL32.dll
 0002:00000078       __imp_QueryPerformanceCounter 0000000180005078     kernel32:KERNEL32.dll
 0002:00000080       __imp_GetCurrentProcessId  0000000180005080     kernel32:KERNEL32.dll
 0002:00000088       __imp_GetCurrentThreadId   0000000180005088     kernel32:KERNEL32.dll
 0002:00000090       __imp_GetSystemTimeAsFileTime 0000000180005090     kernel32:KERNEL32.dll
 0002:00000098       __imp_DisableThreadLibraryCalls 0000000180005098     kernel32:KERNEL32.dll
 0002:000000a0       __imp_InitializeSListHead  00000001800050a0     kernel32:KERNEL32.dll
 0002:000000a8       \177KERNEL32_NULL_THUNK_DATA 00000001800050a8     kernel32:KERNEL32.dll
 0002:000000b0       __imp_memcpy               00000001800050b0     vcruntime:VCRUNTIME140.dll
 0002:000000b8       __imp_memset               00000001800050b8     vcruntime:VCRUNTIME140.dll
 0002:000000c0       __imp_strchr               00000001800050c0     vcruntime:VCRUNTIME140.dll
 0002:000000c8       __imp___C_specific_handler 00000001800050c8     vcruntime:VCRUNTIME140.dll
 0002:000000d0       __imp___std_type_info_destroy_list 00000001800050d0     vcruntime:VCRUNTIME140.dll
 0002:000000d8       \177VCRUNTIME140_NULL_THUNK_DATA 00000001800050d8     vcruntime:VCRUNTIME140.dll
 0002:000000e0       __imp_strtol               00000001800050e0     ucrt:api-ms-win-crt-convert-l1-1-0.dll
 0002:000000e8       \177api-ms-win-crt-convert-l1-1-0_NULL_THUNK_DATA 00000001800050e8     ucrt:api-ms-win-crt-convert-l1-1-0.dll
 0002:000000f0       __imp_malloc               00000001800050f0     ucrt:api-ms-win-crt-heap-l1-1-0.dll
 0002:000000f8       __imp_free                 00000001800050f8     ucrt:api-ms-win-crt-heap-l1-1-0.dll
 0002:00000100       \177api-ms-win-crt-heap-l1-1-0_NULL_THUNK_DATA 0000000180005100     ucrt:api-ms-win-crt-heap-l1-1-0.dll
 0002:00000108       __imp__errno               0000000180005108     ucrt:api-ms-win-crt-runtime-l1-1-0.dll
 0002:00000110       __imp_exit                 0000000180005110     ucrt:api-ms-win-crt-runtime-l1-1-0.dll
 0002:00000118       __imp__cexit               0000000180005118     ucrt:api-ms-win-crt-runtime-l1-1-0.dll
 0002:00000120       __imp__crt_atexit          0000000180005120     ucrt:api-ms-win-crt-runtime-l1-1-0.dll
 0002:00000128       __imp__execute_onexit_table 0000000180005128     ucrt:api-ms-win-crt-runtime-l1-1-0.dll
 0002:00000130       __imp__register_onexit_function 0000000180005130     ucrt:api-ms-win-crt-runtime-l1-1-0.dll
 0002:00000138       __imp__initialize_onexit_table 0000000180005138     ucrt:api-ms-win-crt-runtime-l1-1-0.dll
 0002:00000140       __imp__initialize_narrow_environment 0000000180005140     ucrt:api-ms-win-crt-runtime-l1-1-0.dll
 0002:00000148       __imp__configure_narrow_argv 0000000180005148     ucrt:api-ms-win-crt-runtime-l1-1-0.dll
 0002:00000150       __imp__seh_filter_dll      0000000180005150     ucrt:api-ms-win-crt-runtime-l1-1-0.dll
 0002:00000158       __imp__initterm_e          0000000180005158     ucrt:api-ms-win-crt-runtime-l1-1-0.dll
 0002:00000160       __imp__initterm            0000000180005160     ucrt:api-ms-win-crt-runtime-l1-1-0.dll
 0002:00000168       \177api-ms-win-crt-runtime-l1-1-0_NULL_THUNK_DATA 0000000180005168     ucrt:api-ms-win-crt-runtime-l1-1-0.dll
 0002:00000170       __imp___acrt_iob_func      0000000180005170     ucrt:api-ms-win-crt-stdio-l1-1-0.dll
 0002:00000178       __imp_fflush               0000000180005178     ucrt:api-ms-win-crt-stdio-l1-1-0.dll
 0002:00000180       __imp___stdio_common_vsprintf 0000000180005180     ucrt:api-ms-win-crt-stdio-l1-1-0.dll
 0002:00000188       __imp___stdio_common_vfprintf 0000000180005188     ucrt:api-ms-win-crt-stdio-l1-1-0.dll
 0002:00000190       \177api-ms-win-crt-stdio-l1-1-0_NULL_THUNK_DATA 0000000180005190     ucrt:api-ms-win-crt-stdio-l1-1-0.dll
 0002:00000198       __imp_strcmp               0000000180005198     ucrt:api-ms-win-crt-string-l1-1-0.dll
 0002:000001a0       __imp__strdup              00000001800051a0     ucrt:api-ms-win-crt-string-l1-1-0.dll
 0002:000001a0       __imp_strdup               00000001800051a0     ucrt:api-ms-win-crt-string-l1-1-0.dll
 0002:000001a8       __imp_strlen               00000001800051a8     ucrt:api-ms-win-crt-string-l1-1-0.dll
 0002:000001b0       __imp_strpbrk              00000001800051b0     ucrt:api-ms-win-crt-string-l1-1-0.dll
 0002:000001b8       __imp_strncpy              00000001800051b8     ucrt:api-ms-win-crt-string-l1-1-0.dll
 0002:000001c0       \177api-ms-win-crt-string-l1-1-0_NULL_THUNK_DATA 00000001800051c0     ucrt:api-ms-win-crt-string-l1-1-0.dll
 0002:000001c8       __guard_check_icall_fptr   00000001800051c8     MSVCRT:guard_support.obj
 0002:000001d0       __guard_xfg_check_icall_fptr 00000001800051d0     MSVCRT:guard_support.obj
 0002:000001d8       __guard_dispatch_icall_fptr 00000001800051d8     MSVCRT:guard_support.obj
 0002:000001e0       __guard_xfg_dispatch_icall_fptr 00000001800051e0     MSVCRT:guard_support.obj
 0002:000001e8       __guard_xfg_table_dispatch_icall_fptr 00000001800051e8     MSVCRT:guard_support.obj
 0002:000001f0       __castguard_check_failure_os_handled_fptr 00000001800051f0     MSVCRT:guard_support.obj
 0002:000001f8       __guard_memcpy_fptr        00000001800051f8     vcruntime:softmemtag.obj
 0002:00000200       __xc_a                     0000000180005200     MSVCRT:initializers.obj
 0002:00000208       __xc_z                     0000000180005208     MSVCRT:initializers.obj
 0002:00000210       __xi_a                     0000000180005210     MSVCRT:initializers.obj
 0002:00000220       __xi_z                     0000000180005220     MSVCRT:initializers.obj
 0002:00000228       __xl_a                     0000000180005228     MSVCRT:tlssup.obj
 0002:00000230       __xl_z                     0000000180005230     MSVCRT:tlssup.obj
 0002:00000238       __xp_a                     0000000180005238     MSVCRT:initializers.obj
 0002:00000240       __xp_z                     0000000180005240     MSVCRT:initializers.obj
 0002:00000248       __xt_a                     0000000180005248     MSVCRT:initializers.obj
 0002:00000250       __xt_z                     0000000180005250     MSVCRT:initializers.obj
 0002:00000260       g_refKindStr               0000000180005260     libsystemclssearch_agent.obj
 0002:00000420       ??_C@_09BPLDFGCI@unknown_0@ 0000000180005420     libsystemclssearch_agent.obj
 0002:00000430       ??_C@_0BL@FPNMECJD@JVMTI_HEAP_REFERENCE_CLASS@ 0000000180005430     libsystemclssearch_agent.obj
 0002:00000450       ??_C@_0BL@FKGKKLNM@JVMTI_HEAP_REFERENCE_FIELD@ 0000000180005450     libsystemclssearch_agent.obj
 0002:00000470       ??_C@_0CD@CAEHCFJF@JVMTI_HEAP_REFERENCE_ARRAY_ELEM@ 0000000180005470     libsystemclssearch_agent.obj
 0002:00000498       ??_C@_0CC@DNEBMCNK@JVMTI_HEAP_REFERENCE_CLASS_LOAD@ 0000000180005498     libsystemclssearch_agent.obj
 0002:000004c0       ??_C@_0BN@CJMIPEBB@JVMTI_HEAP_REFERENCE_SIGNERS@ 00000001800054c0     libsystemclssearch_agent.obj
 0002:000004e0       ??_C@_0CH@HBOIDPEB@JVMTI_HEAP_REFERENCE_PROTECTION@ 00000001800054e0     libsystemclssearch_agent.obj
 0002:00000508       ??_C@_0BP@MDKGDGKL@JVMTI_HEAP_REFERENCE_INTERFACE@ 0000000180005508     libsystemclssearch_agent.obj
 0002:00000528       ??_C@_0CC@JJMIHNJH@JVMTI_HEAP_REFERENCE_STATIC_FIE@ 0000000180005528     libsystemclssearch_agent.obj
 0002:00000550       ??_C@_0CD@IDHEEGID@JVMTI_HEAP_REFERENCE_CONSTANT_P@ 0000000180005550     libsystemclssearch_agent.obj
 0002:00000578       ??_C@_0CA@EFFCHNG@JVMTI_HEAP_REFERENCE_SUPERCLASS@ 0000000180005578     libsystemclssearch_agent.obj
 0002:00000598       ??_C@_0L@PCDFHGCJ@unknown_11@ 0000000180005598     libsystemclssearch_agent.obj
 0002:000005a8       ??_C@_0L@NJBICFOK@unknown_12@ 00000001800055a8     libsystemclssearch_agent.obj
 0002:000005b8       ??_C@_0L@MAADBEKL@unknown_13@ 00000001800055b8     libsystemclssearch_agent.obj
 0002:000005c8       ??_C@_0L@IPECICGM@unknown_14@ 00000001800055c8     libsystemclssearch_agent.obj
 0002:000005d8       ??_C@_0L@JGFJLDCN@unknown_15@ 00000001800055d8     libsystemclssearch_agent.obj
 0002:000005e8       ??_C@_0L@LNHEOAOO@unknown_16@ 00000001800055e8     libsystemclssearch_agent.obj
 0002:000005f8       ??_C@_0L@KEGPNBKP@unknown_17@ 00000001800055f8     libsystemclssearch_agent.obj
 0002:00000608       ??_C@_0L@CDPHMNGA@unknown_18@ 0000000180005608     libsystemclssearch_agent.obj
 0002:00000618       ??_C@_0L@DKOMPMCB@unknown_19@ 0000000180005618     libsystemclssearch_agent.obj
 0002:00000628       ??_C@_0L@OJGIPJDB@unknown_20@ 0000000180005628     libsystemclssearch_agent.obj
 0002:00000638       ??_C@_0CA@KAOFNDEM@JVMTI_HEAP_REFERENCE_JNI_GLOBAL@ 0000000180005638     libsystemclssearch_agent.obj
 0002:00000658       ??_C@_0CC@HPFAJBK@JVMTI_HEAP_REFERENCE_SYSTEM_CLA@ 0000000180005658     libsystemclssearch_agent.obj
 0002:00000680       ??_C@_0BN@FDEGFOHC@JVMTI_HEAP_REFERENCE_MONITOR@ 0000000180005680     libsystemclssearch_agent.obj
 0002:000006a0       ??_C@_0CB@HKIBCMAJ@JVMTI_HEAP_REFERENCE_STACK_LOCA@ 00000001800056a0     libsystemclssearch_agent.obj
 0002:000006c8       ??_C@_0BP@EAACMMOE@JVMTI_HEAP_REFERENCE_JNI_LOCAL@ 00000001800056c8     libsystemclssearch_agent.obj
 0002:000006e8       ??_C@_0BM@IJDEOGOE@JVMTI_HEAP_REFERENCE_THREAD@ 00000001800056e8     libsystemclssearch_agent.obj
 0002:00000708       ??_C@_0BL@EDGPPKC@JVMTI_HEAP_REFERENCE_OTHER@ 0000000180005708     libsystemclssearch_agent.obj
 0002:00000724       ??_C@_04BCJPDBDA@Code@     0000000180005724     libsystemclssearch_agent.obj
 0002:00000730       ??_C@_0BA@OCLMCFKC@LineNumberTable@ 0000000180005730     libsystemclssearch_agent.obj
 0002:00000740       ??_C@_0BD@CPAEPILC@LocalVariableTable@ 0000000180005740     libsystemclssearch_agent.obj
 0002:00000758       ??_C@_0BH@NMBDNHBD@LocalVariableTypeTable@ 0000000180005758     libsystemclssearch_agent.obj
 0002:00000770       ??_C@_0O@HIHEEDNJ@StackMapTable@ 0000000180005770     libsystemclssearch_agent.obj
 0002:00000780       ??_C@_0L@HCDIAMJG@?9?5?$CFs?0?5?$CFd?3?5@ 0000000180005780     libsystemclssearch_agent.obj
 0002:00000790       ??_C@_0JI@HLPECLFI@?$CD?5?4?4?4?6?$CD?5ERROR?3?5too?5many?5complai@ 0000000180005790     libsystemclssearch_agent.obj
 0002:00000830       ??_C@_0ED@JNEKCCOB@The?5following?5fake?5exception?5st@ 0000000180005830     libsystemclssearch_agent.obj
 0002:00000878       ??_C@_0CN@FCNMDFBH@nsk?4share?4Fake_Exception_for_RU@ 0000000180005878     libsystemclssearch_agent.obj
 0002:000008a8       ??_C@_08PGFFNAEI@?$CI?$CFs?3?$CFd?$CJ?5@ 00000001800058a8     libsystemclssearch_agent.obj
 0002:000008b8       ??_C@_0DP@IENMAEGI@s?2test?2hotspot?2jtreg?2vmTestbase@ 00000001800058b8     libsystemclssearch_agent.obj
 0002:000008f8       ??_C@_0BL@NDJLFFJB@?7at?5nsk_lvcomplain?$CI?$CFs?3?$CFd?$CJ?6@ 00000001800058f8     libsystemclssearch_agent.obj
 0002:00000918       ??_C@_0BC@JOOKAFKF@?$CD?5ERROR?3?5?$CFs?0?5?$CFd?3?5@ 0000000180005918     libsystemclssearch_agent.obj
 0002:00000930       ??_C@_09KJEAHMEH@?$CD?5ERROR?3?5@ 0000000180005930     libsystemclssearch_agent.obj
 0002:0000093c       ??_C@_02GPIOPFAK@?$DO?$DO@ 000000018000593c     libsystemclssearch_agent.obj
 0002:00000940       ??_C@_02FODMEDOG@?$DM?$DM@ 0000000180005940     libsystemclssearch_agent.obj
 0002:00000944       ??_C@_02DJGKEECL@?4?4@     0000000180005944     libsystemclssearch_agent.obj
 0002:00000948       ??_C@_0O@CJPGJOAF@?9?5?$CFs?0?5?$CFd?3?5?$CFs?5@ 0000000180005948     libsystemclssearch_agent.obj
 0002:00000958       ??_C@_0CB@IAKPDOIC@?$CD?5?5?5verified?5assertion?5is?5FALSE@ 0000000180005958     libsystemclssearch_agent.obj
 0002:00000980       ??_C@_0CO@LGONDEPD@stdout?3?5fflush?5failed?5?9?5err?$DN?$CFd?5@ 0000000180005980     libsystemclssearch_agent.obj
 0002:000009b0       ??_C@_0CO@KBGKJPBD@stderr?3?5fflush?5failed?5?9?5err?$DN?$CFd?5@ 00000001800059b0     libsystemclssearch_agent.obj
 0002:000009de       ??_C@_00CNPNBAHC@@         00000001800059de     libsystemclssearch_agent.obj
 0002:000009e0       ??_C@_0BB@JCNMKLLK@JVMTI_ERROR_NONE@ 00000001800059e0     libsystemclssearch_agent.obj
 0002:000009f8       ??_C@_0BL@LDIMKLPH@JVMTI_ERROR_INVALID_THREAD@ 00000001800059f8     libsystemclssearch_agent.obj
 0002:00000a18       ??_C@_0CB@PJFPAIKJ@JVMTI_ERROR_INVALID_THREAD_GROU@ 0000000180005a18     libsystemclssearch_agent.obj
 0002:00000a40       ??_C@_0BN@LLMKHMNF@JVMTI_ERROR_INVALID_PRIORITY@ 0000000180005a40     libsystemclssearch_agent.obj
 0002:00000a60       ??_C@_0CB@MBOFKAGB@JVMTI_ERROR_THREAD_NOT_SUSPENDE@ 0000000180005a60     libsystemclssearch_agent.obj
 0002:00000a88       ??_C@_0BN@FABOLPBI@JVMTI_ERROR_THREAD_SUSPENDED@ 0000000180005a88     libsystemclssearch_agent.obj
 0002:00000aa8       ??_C@_0BN@FDGNOBJM@JVMTI_ERROR_THREAD_NOT_ALIVE@ 0000000180005aa8     libsystemclssearch_agent.obj
 0002:00000ac8       ??_C@_0BL@GOBIFKNJ@JVMTI_ERROR_INVALID_OBJECT@ 0000000180005ac8     libsystemclssearch_agent.obj
 0002:00000ae8       ??_C@_0BK@FCMAJPPC@JVMTI_ERROR_INVALID_CLASS@ 0000000180005ae8     libsystemclssearch_agent.obj
 0002:00000b08       ??_C@_0BP@IKLLBKEB@JVMTI_ERROR_CLASS_NOT_PREPARED@ 0000000180005b08     libsystemclssearch_agent.obj
 0002:00000b28       ??_C@_0BN@KLPPLKG@JVMTI_ERROR_INVALID_METHODID@ 0000000180005b28     libsystemclssearch_agent.obj
 0002:00000b48       ??_C@_0BN@BCEKOKND@JVMTI_ERROR_INVALID_LOCATION@ 0000000180005b48     libsystemclssearch_agent.obj
 0002:00000b68       ??_C@_0BM@DFDGPME@JVMTI_ERROR_INVALID_FIELDID@ 0000000180005b68     libsystemclssearch_agent.obj
 0002:00000b88       ??_C@_0BL@NELIEPEC@JVMTI_ERROR_NO_MORE_FRAMES@ 0000000180005b88     libsystemclssearch_agent.obj
 0002:00000ba8       ??_C@_0BJ@BDBECFDM@JVMTI_ERROR_OPAQUE_FRAME@ 0000000180005ba8     libsystemclssearch_agent.obj
 0002:00000bc8       ??_C@_0BK@MIIFNLOB@JVMTI_ERROR_TYPE_MISMATCH@ 0000000180005bc8     libsystemclssearch_agent.obj
 0002:00000be8       ??_C@_0BJ@HPCAOILC@JVMTI_ERROR_INVALID_SLOT@ 0000000180005be8     libsystemclssearch_agent.obj
 0002:00000c08       ??_C@_0BG@CHILOPNI@JVMTI_ERROR_DUPLICATE@ 0000000180005c08     libsystemclssearch_agent.obj
 0002:00000c20       ??_C@_0BG@DIEMLHKM@JVMTI_ERROR_NOT_FOUND@ 0000000180005c20     libsystemclssearch_agent.obj
 0002:00000c38       ??_C@_0BM@NHMCKHOB@JVMTI_ERROR_INVALID_MONITOR@ 0000000180005c38     libsystemclssearch_agent.obj
 0002:00000c58       ??_C@_0BO@PPEDAJGL@JVMTI_ERROR_NOT_MONITOR_OWNER@ 0000000180005c58     libsystemclssearch_agent.obj
 0002:00000c78       ??_C@_0BG@FCAIPEID@JVMTI_ERROR_INTERRUPT@ 0000000180005c78     libsystemclssearch_agent.obj
 0002:00000c90       ??_C@_0CB@EGDBNKOI@JVMTI_ERROR_INVALID_CLASS_FORMA@ 0000000180005c90     libsystemclssearch_agent.obj
 0002:00000cb8       ??_C@_0CG@DGKOGIAL@JVMTI_ERROR_CIRCULAR_CLASS_DEFI@ 0000000180005cb8     libsystemclssearch_agent.obj
 0002:00000ce0       ??_C@_0BP@ICEALPKC@JVMTI_ERROR_FAILS_VERIFICATION@ 0000000180005ce0     libsystemclssearch_agent.obj
 0002:00000d00       ??_C@_0DC@JDACLMIO@JVMTI_ERROR_UNSUPPORTED_REDEFIN@ 0000000180005d00     libsystemclssearch_agent.obj
 0002:00000d38       ??_C@_0DE@GKDKNOMJ@JVMTI_ERROR_UNSUPPORTED_REDEFIN@ 0000000180005d38     libsystemclssearch_agent.obj
 0002:00000d70       ??_C@_0BO@LAFKIOG@JVMTI_ERROR_INVALID_TYPESTATE@ 0000000180005d70     libsystemclssearch_agent.obj
 0002:00000d90       ??_C@_0DH@INDGCLLB@JVMTI_ERROR_UNSUPPORTED_REDEFIN@ 0000000180005d90     libsystemclssearch_agent.obj
 0002:00000dc8       ??_C@_0DE@NHEOMMGI@JVMTI_ERROR_UNSUPPORTED_REDEFIN@ 0000000180005dc8     libsystemclssearch_agent.obj
 0002:00000e00       ??_C@_0CA@EKPNJOEP@JVMTI_ERROR_UNSUPPORTED_VERSION@ 0000000180005e00     libsystemclssearch_agent.obj
 0002:00000e20       ??_C@_0BN@OFFMAHHL@JVMTI_ERROR_NAMES_DONT_MATCH@ 0000000180005e20     libsystemclssearch_agent.obj
 0002:00000e40       ??_C@_0DN@HHBBLAKE@JVMTI_ERROR_UNSUPPORTED_REDEFIN@ 0000000180005e40     libsystemclssearch_agent.obj
 0002:00000e80       ??_C@_0DO@HMBGBGNA@JVMTI_ERROR_UNSUPPORTED_REDEFIN@ 0000000180005e80     libsystemclssearch_agent.obj
 0002:00000ec0       ??_C@_0BP@PBECGKHJ@JVMTI_ERROR_UNMODIFIABLE_CLASS@ 0000000180005ec0     libsystemclssearch_agent.obj
 0002:00000ee0       ??_C@_0BK@CANILEHF@JVMTI_ERROR_NOT_AVAILABLE@ 0000000180005ee0     libsystemclssearch_agent.obj
 0002:00000f00       ??_C@_0CE@INJKMEFK@JVMTI_ERROR_MUST_POSSESS_CAPABI@ 0000000180005f00     libsystemclssearch_agent.obj
 0002:00000f28       ??_C@_0BJ@LBFPFPDM@JVMTI_ERROR_NULL_POINTER@ 0000000180005f28     libsystemclssearch_agent.obj
 0002:00000f48       ??_C@_0BP@CHJPNNEM@JVMTI_ERROR_ABSENT_INFORMATION@ 0000000180005f48     libsystemclssearch_agent.obj
 0002:00000f68       ??_C@_0BP@OMFMNLC@JVMTI_ERROR_INVALID_EVENT_TYPE@ 0000000180005f68     libsystemclssearch_agent.obj
 0002:00000f88       ??_C@_0BN@BIBNPHHO@JVMTI_ERROR_ILLEGAL_ARGUMENT@ 0000000180005f88     libsystemclssearch_agent.obj
 0002:00000fa8       ??_C@_0BK@KKNDHDCE@JVMTI_ERROR_NATIVE_METHOD@ 0000000180005fa8     libsystemclssearch_agent.obj
 0002:00000fc8       ??_C@_0BK@PMKCFHAE@JVMTI_ERROR_OUT_OF_MEMORY@ 0000000180005fc8     libsystemclssearch_agent.obj
 0002:00000fe8       ??_C@_0BK@NNJBDMNB@JVMTI_ERROR_ACCESS_DENIED@ 0000000180005fe8     libsystemclssearch_agent.obj
 0002:00001008       ??_C@_0BI@GHECLMNC@JVMTI_ERROR_WRONG_PHASE@ 0000000180006008     libsystemclssearch_agent.obj
 0002:00001020       ??_C@_0BF@OLIHJOII@JVMTI_ERROR_INTERNAL@ 0000000180006020     libsystemclssearch_agent.obj
 0002:00001038       ??_C@_0BO@EOHGKJHI@JVMTI_ERROR_UNATTACHED_THREAD@ 0000000180006038     libsystemclssearch_agent.obj
 0002:00001058       ??_C@_0CA@LKHFDACL@JVMTI_ERROR_INVALID_ENVIRONMENT@ 0000000180006058     libsystemclssearch_agent.obj
 0002:00001078       ??_C@_0BA@MMFHLOKK@?$DMunknown?5error?$DO@ 0000000180006078     libsystemclssearch_agent.obj
 0002:00001088       ??_C@_0CF@CBHOKDB@throwable?5?$DN?5jni?9?$DOExceptionOccur@ 0000000180006088     libsystemclssearch_agent.obj
 0002:000010b0       ??_C@_03OFAPEBGM@?$CFs?6@  00000001800060b0     libsystemclssearch_agent.obj
 0002:000010b8       ??_C@_0DM@LPIGEGNJ@s?2test?2hotspot?2jtreg?2vmTestbase@ 00000001800060b8     libsystemclssearch_agent.obj
 0002:000010f8       ??_C@_0CC@NFCNPEPK@Exception?5in?5JNI?5call?5?$CIcleared?$CJ@ 00000001800060f8     libsystemclssearch_agent.obj
 0002:00001120       ??_C@_0BJ@IBAKFIKF@jni?9?$DOExceptionDescribe?$CI?$CJ@ 0000000180006120     libsystemclssearch_agent.obj
 0002:00001140       ??_C@_0BG@GGKALKMH@jni?9?$DOExceptionClear?$CI?$CJ@ 0000000180006140     libsystemclssearch_agent.obj
 0002:00001158       ??_C@_0CF@JMGFGJLJ@?$CD?5?5?5verified?5JNI?5assertion?5is?5F@ 0000000180006158     libsystemclssearch_agent.obj
 0002:00001180       ??_C@_07KBAMPNJK@verbose@  0000000180006180     libsystemclssearch_agent.obj
 0002:00001188       ??_C@_0DN@PKJBOLAP@nsk_jvmti_parseOptions?$CI?$CJ?3?5unexp@ 0000000180006188     libsystemclssearch_agent.obj
 0002:000011c8       ??_C@_05IMBNNINJ@trace@    00000001800061c8     libsystemclssearch_agent.obj
 0002:000011d0       ??_C@_0DD@BJKGNDMB@nsk_jvmti_parseOptions?$CI?$CJ?3?5no?5va@ 00000001800061d0     libsystemclssearch_agent.obj
 0002:00001204       ??_C@_04CGFJFPFD@none@     0000000180006204     libsystemclssearch_agent.obj
 0002:0000120c       ??_C@_06BMELKFMA@before@   000000018000620c     libsystemclssearch_agent.obj
 0002:00001214       ??_C@_05CMKPCFDK@after@    0000000180006214     libsystemclssearch_agent.obj
 0002:0000121c       ??_C@_03NFKEKGGK@all@      000000018000621c     libsystemclssearch_agent.obj
 0002:00001220       ??_C@_0DM@NDNJGJKE@nsk_jvmti_parseOptions?$CI?$CJ?3?5uexpe@ 0000000180006220     libsystemclssearch_agent.obj
 0002:00001260       ??_C@_08NBBJKJO@waittime@  0000000180006260     libsystemclssearch_agent.obj
 0002:00001270       ??_C@_0DO@CMHGAOHC@nsk_jvmti_parseOptions?$CI?$CJ?3?5not?5i@ 0000000180006270     libsystemclssearch_agent.obj
 0002:000012b0       ??_C@_0DL@LNMPBDLN@nsk_jvmti_parseOptions?$CI?$CJ?3?5negat@ 00000001800062b0     libsystemclssearch_agent.obj
 0002:000012f0       ??_C@_0DA@GMFJNOJH@nsk_jvmti_parseOptions?$CI?$CJ?3?5unkno@ 00000001800062f0     libsystemclssearch_agent.obj
 0002:00001320       ??_C@_0CO@CCIAMEAN@nsk_jvmti_parseOptions?$CI?$CJ?3?5found@ 0000000180006320     libsystemclssearch_agent.obj
 0002:00001350       ??_C@_0CJ@OEGPCGDL@nsk_jvmti_parseOptions?$CI?$CJ?3?5out?5o@ 0000000180006350     libsystemclssearch_agent.obj
 0002:00001380       ??_C@_0DI@NMBHPGGF@nsk_jvmti_parseOptions?$CI?$CJ?3?5too?5m@ 0000000180006380     libsystemclssearch_agent.obj
 0002:000013b8       ??_C@_03POGCGECB@?5?0?$HO@ 00000001800063b8     libsystemclssearch_agent.obj
 0002:000013c0       ??_C@_0DC@GKLNPJIJ@nsk_jvmti_findOptionValue?$CI?$CJ?3?5op@ 00000001800063c0     libsystemclssearch_agent.obj
 0002:000013f8       ??_C@_0DI@KBNKFNAE@nsk_jvmti_findOptionStringValue@ 00000001800063f8     libsystemclssearch_agent.obj
 0002:00001430       ??_C@_0EB@JFLDPDIF@nsk_jvmti_findOptionStringValue@ 0000000180006430     libsystemclssearch_agent.obj
 0002:00001478       ??_C@_0CB@MLNJNCLJ@?5?5jvmti?5error?3?5code?$DN?$CFd?0?5name?$DN?$CFs@ 0000000180006478     libsystemclssearch_agent.obj
 0002:000014a0       ??_C@_0CD@OHBGDKMK@?$CD?5?5?5jvmti?5error?3?5code?$DN?$CFd?0?5name?$DN@ 00000001800064a0     libsystemclssearch_agent.obj
 0002:000014c8       ??_C@_0CG@JNNCGPHB@?$CD?5?5?5error?5expected?3?5code?$DN?$CFd?0?5na@ 00000001800064c8     libsystemclssearch_agent.obj
 0002:000014f0       ??_C@_0EB@IMGKPCGE@?$CIstr_obj?5?$DN?5jni?9?$DONewStringUTF?$CIco@ 00000001800064f0     libsystemclssearch_agent.obj
 0002:00001540       ??_C@_0EA@HFOGGBCC@s?2test?2hotspot?2jtreg?2vmTestbase@ 0000000180006540     libsystemclssearch_agent.obj
 0002:00001580       ??_C@_05KKCIMGE@error@     0000000180006580     libsystemclssearch_agent.obj
 0002:00001588       ??_C@_0CJ@JACLEAA@Test?5failed?5by?5setFailStatus?$CI?$CJ?4@ 0000000180006588     libsystemclssearch_agent.obj
 0002:000015b8       ??_C@_0BD@HGNAOMCP@agent_data_monitor@ 00000001800065b8     libsystemclssearch_agent.obj
 0002:000015d0       ??_C@_0EB@OGCLGKLN@javaVM?9?$DOGetEnv?$CI?$CIvoid?5?$CK?$CK?$CJ?$CGjvmti_@ 00000001800065d0     libsystemclssearch_agent.obj
 0002:00001620       ??_C@_0EA@PNBCDMOA@s?2test?2hotspot?2jtreg?2vmTestbase@ 0000000180006620     libsystemclssearch_agent.obj
 0002:00001660       ??_C@_0CI@DDPIFBGM@init_agent_data?$CIjvmti_env?0?5?$CGage@ 0000000180006660     libsystemclssearch_agent.obj
 0002:00001688       ??_C@_0DI@ILAHDLMP@?$CI?$CKagentThreadProc?$CJ?$CIjvmti_env?0?5a@ 0000000180006688     libsystemclssearch_agent.obj
 0002:000016c0       ??_C@_0BD@KDBALNLB@JVMTI?5agent?5thread@ 00000001800066c0     libsystemclssearch_agent.obj
 0002:000016d8       ??_C@_0BB@NOKBFPFO@java?1lang?1Thread@ 00000001800066d8     libsystemclssearch_agent.obj
 0002:000016ec       ??_C@_06FALKBLGB@?$DMinit?$DO@ 00000001800066ec     libsystemclssearch_agent.obj
 0002:000016f8       ??_C@_0BG@IKDDPPGD@?$CILjava?1lang?1String?$DL?$CJV@ 00000001800066f8     libsystemclssearch_agent.obj
 0002:00001710       ??_C@_0EB@IFJBFEKC@?$CIthreadClass?5?$DN?5jni_env?9?$DOFindCla@ 0000000180006710     libsystemclssearch_agent.obj
 0002:00001760       ??_C@_0GF@FGFIBKKL@?$CIthreadCtor?5?$DN?5jni_env?9?$DOGetMetho@ 0000000180006760     libsystemclssearch_agent.obj
 0002:000017c8       ??_C@_0DN@NCPDJLOG@?$CIthreadName?5?$DN?5jni_env?9?$DONewStrin@ 00000001800067c8     libsystemclssearch_agent.obj
 0002:00001810       ??_C@_0FE@PFKODBGC@?$CIthreadObject?5?$DN?5jni_env?9?$DONewObj@ 0000000180006810     libsystemclssearch_agent.obj
 0002:00001870       ??_C@_0ED@HOBAHHJI@?$CIthreadGlobalRef?5?$DN?5jni_env?9?$DONew@ 0000000180006870     libsystemclssearch_agent.obj
 0002:000018c0       ??_C@_0FN@HNJJAHFC@jvmti_env?9?$DORunAgentThread?$CIagent@ 00000001800068c0     libsystemclssearch_agent.obj
 0002:00001920       ??_C@_0EA@MOJDNKDF@Debuggee?5status?5sync?5aborted?5be@ 0000000180006920     libsystemclssearch_agent.obj
 0002:00001960       ??_C@_0EA@EEOEJAEN@status?5?$DN?5syncDebuggeeStatus?$CIjni@ 0000000180006960     libsystemclssearch_agent.obj
 0002:000019a0       ??_C@_0BL@JBCFNBMB@nsk_jvmti_resetAgentData?$CI?$CJ@ 00000001800069a0     libsystemclssearch_agent.obj
 0002:000019c0       ??_C@_0DN@NNGECJON@jvmti_env?9?$DOSetEventNotification@ 00000001800069c0     libsystemclssearch_agent.obj
 0002:00001a00       ??_C@_0EL@LPBEELIP@s?2test?2hotspot?2jtreg?2vmTestbase@ 0000000180006a00     libsystemclssearch_agent.obj
 0002:00001a50       ??_C@_0CK@JDAMFDMJ@jvmti?9?$DOSetTag?$CIo?0?5tag?$CJ?5?$DN?$DN?5JVMTI_@ 0000000180006a50     libsystemclssearch_agent.obj
 0002:00001a80       ??_C@_0CC@DAMNHKNI@Can?8t?5set?5tag?5?$CFli?5for?5object?5?$CFl@ 0000000180006a80     libsystemclssearch_agent.obj
 0002:00001aa8       ??_C@_0DL@HAJPNKEF@jvmti?9?$DOGetObjectHashCode?$CIo?0?5?$CGha@ 0000000180006aa8     libsystemclssearch_agent.obj
 0002:00001ae8       ??_C@_0BL@JFPIEOBF@Can?8t?5get?5hash?5object?5?$CFlx?6@ 0000000180006ae8     libsystemclssearch_agent.obj
 0002:00001b08       ??_C@_0BG@DICPHBKN@setTag?3?5?$CF08x?5?$DM?9?5?$CF?53li@ 0000000180006b08     libsystemclssearch_agent.obj
 0002:00001b20       ??_C@_0DH@FCEEBDMJ@?$CIs?5?$DN?5jni?9?$DOGetStringUTFChars?$CIsIn@ 0000000180006b20     libsystemclssearch_agent.obj
 0002:00001b58       ??_C@_0BJ@OKKGHDCN@Can?8t?5get?5string?5at?5?$CF?$CDp?6@ 0000000180006b58     libsystemclssearch_agent.obj
 0002:00001b78       ??_C@_0BP@EKFLGGFJ@Can?8t?5get?5string?5at?5?$CF?$CDp?3?5null?6@ 0000000180006b78     libsystemclssearch_agent.obj
 0002:00001b98       ??_C@_06ICODBHCL@?5?1?1?5?$CFs@ 0000000180006b98     libsystemclssearch_agent.obj
 0002:00001ba0       ??_C@_0DB@KGFPLEGO@?$CIr?5?$DN?5jvmti?9?$DOGetTag?$CIo?0?5?$CGtag?$CJ?$CJ?5?$DN?$DN@ 0000000180006ba0     libsystemclssearch_agent.obj
 0002:00001bd8       ??_C@_0CO@PDAGBCGJ@Can?8t?5GetTag?5for?5object?5?$CFlx?4?5Re@ 0000000180006bd8     libsystemclssearch_agent.obj
 0002:00001c08       ??_C@_0CH@HPEODOHC@TEST_BUG?3?5Max?4?5number?5of?5refs?5r@ 0000000180006c08     libsystemclssearch_agent.obj
 0002:00001c30       ??_C@_0DI@PHFCABIM@?$CIr?5?$DN?5jvmti?9?$DOGetTag?$CIfrom?0?5?$CGtagFr@ 0000000180006c30     libsystemclssearch_agent.obj
 0002:00001c68       ??_C@_0DI@MDEGFNKD@TEST_BUG?3?5Can?8t?5GetTag?5for?5obje@ 0000000180006c68     libsystemclssearch_agent.obj
 0002:00001ca0       ??_C@_0DE@MLELJAHM@?$CIr?5?$DN?5jvmti?9?$DOGetTag?$CIto?0?5?$CGtagTo?$CJ?$CJ@ 0000000180006ca0     libsystemclssearch_agent.obj
 0002:00001cd4       ??_C@_04LKCODBAO@tmp?1@    0000000180006cd4     libsystemclssearch_agent.obj
 0002:00001ce0       ??_C@_0BD@PNDFDFAN@Add?5segment?3?5?$CC?$CFs?$CC?6@ 0000000180006ce0     libsystemclssearch_agent.obj
 0002:00001d00       ??_C@_0GH@LCKDHMDL@s?2test?2hotspot?2jtreg?2vmTestbase@ 0000000180006d00     libsystemclssearch_agent.obj
 0002:00001d68       ??_C@_0CN@JLILJNGP@jvmti?9?$DOAddToSystemClassLoaderSe@ 0000000180006d68     libsystemclssearch_agent.obj
 0002:00001d98       ??_C@_0CI@PKNHJJPM@TEST?5FAILURE?3?5failed?5to?5add?5seg@ 0000000180006d98     libsystemclssearch_agent.obj
 0002:00001dc0       ??_C@_0N@GCANCHC@?5?5?4?4?4?5added?6@ 0000000180006dc0     libsystemclssearch_agent.obj
 0002:00001dd0       ??_C@_0BL@EMFDJAKL@Add?5illegal?5segment?3?5?$CC?$CFs?$CC?6@ 0000000180006dd0     libsystemclssearch_agent.obj
 0002:00001df0       ??_C@_0FA@MNIKGOIN@TEST?5FAILURE?3?5got?5wrong?5error?5w@ 0000000180006df0     libsystemclssearch_agent.obj
 0002:00001e40       ??_C@_0BB@CAMEJFFA@?5?5?4?4?4?5not?5added?6@ 0000000180006e40     libsystemclssearch_agent.obj
 0002:00001e60       ??_C@_0EN@NLLKPGNF@?$DO?$DO?$DO?5Testcase?5?$CD1?3?5Add?5bootstrap?5@ 0000000180006e60     libsystemclssearch_agent.obj
 0002:00001eb0       ??_C@_08ELCMPAFF@VMInit?$CI?$CJ@ 0000000180006eb0     libsystemclssearch_agent.obj
 0002:00001ec0       ??_C@_0BI@LJPGANNB@jvmti?9?$DOGetPhase?$CI?$CGphase?$CJ@ 0000000180006ec0     libsystemclssearch_agent.obj
 0002:00001ed8       ??_C@_0CD@HNPPKPIP@TEST?5FAILURE?3?5unable?5to?5get?5pha@ 0000000180006ed8     libsystemclssearch_agent.obj
 0002:00001f00       ??_C@_0BK@CINOGBLO@phase?5?$DN?$DN?5JVMTI_PHASE_LIVE@ 0000000180006f00     libsystemclssearch_agent.obj
 0002:00001f20       ??_C@_0EO@ODEMMFHH@?$DO?$DO?$DO?5Testcase?5?$CD1?3?5Add?5bootstrap?5@ 0000000180006f20     libsystemclssearch_agent.obj
 0002:00001f70       ??_C@_09LAILOHCM@VMDeath?$CI?$CJ@ 0000000180006f70     libsystemclssearch_agent.obj
 0002:00001f80       ??_C@_0CA@MNKGCBCG@nsk_jvmti_parseOptions?$CIoptions?$CJ@ 0000000180006f80     libsystemclssearch_agent.obj
 0002:00001fa0       ??_C@_08KNCGGLEC@segment1@ 0000000180006fa0     libsystemclssearch_agent.obj
 0002:00001fb0       ??_C@_0BG@OFJODEAO@p_segment1?5?$CB?$DN?5nullptr@ 0000000180006fb0     libsystemclssearch_agent.obj
 0002:00001fc8       ??_C@_08IGALDIIB@segment2@ 0000000180006fc8     libsystemclssearch_agent.obj
 0002:00001fd8       ??_C@_0DN@MIAMNFPH@?$CIjvmti?5?$DN?5nsk_jvmti_createJVMTIE@ 0000000180006fd8     libsystemclssearch_agent.obj
 0002:00002018       ??_C@_0N@EMFHEOLN@phasetocheck@ 0000000180007018     libsystemclssearch_agent.obj
 0002:00002028       ??_C@_0BK@LBDCKLBN@phase_to_check?5?$CB?$DN?5nullptr@ 0000000180007028     libsystemclssearch_agent.obj
 0002:00002044       ??_C@_06FKJAAAAK@onload@   0000000180007044     libsystemclssearch_agent.obj
 0002:0000204c       ??_C@_04GLMHKBCH@live@     000000018000704c     libsystemclssearch_agent.obj
 0002:00002060       ??_C@_0EF@IEHDNLE@?$DO?$DO?$DO?5Testcase?5?$CD1?3?5Add?5bootstrap?5@ 0000000180007060     libsystemclssearch_agent.obj
 0002:000020a8       ??_C@_0P@LKCKDJEM@Agent_OnLoad?$CI?$CJ@ 00000001800070a8     libsystemclssearch_agent.obj
 0002:000020b8       ??_C@_0BC@OJMCHGIA@VM_INIT?0?5VM_DEATH@ 00000001800070b8     libsystemclssearch_agent.obj
 0002:000020d0       ??_C@_0BN@MOBPDDBP@Set?5callback?5for?5events?3?5?$CFs?6@ 00000001800070d0     libsystemclssearch_agent.obj
 0002:000020f0       ??_C@_0EC@ODFGFOAJ@jvmti?9?$DOSetEventCallbacks?$CI?$CGevent@ 00000001800070f0     libsystemclssearch_agent.obj
 0002:00002138       ??_C@_0L@HIMFBJJO@?5?5?4?4?4?5set?6@ 0000000180007138     libsystemclssearch_agent.obj
 0002:00002148       ??_C@_0BD@PBPNNGPC@Enable?5events?3?5?$CFs?6@ 0000000180007148     libsystemclssearch_agent.obj
 0002:00002160       ??_C@_0GC@OGFPMMAC@nsk_jvmti_enableEvents?$CI?5JVMTI_E@ 0000000180007160     libsystemclssearch_agent.obj
 0002:000021c8       ??_C@_0P@BAMBNLJF@?5?5?4?4?4?5enabled?6@ 00000001800071c8     libsystemclssearch_agent.obj
 0002:000021f0       ??_C@_1EC@JIJBPKFM@?$AAa?$AAp?$AAi?$AA?9?$AAm?$AAs?$AA?9?$AAw?$AAi?$AAn?$AA?9?$AAc?$AAo?$AAr?$AAe@ 00000001800071f0     MSVCRT:thread_safe_statics.obj
 0002:00002238       ??_C@_1BK@MGMFAEKH@?$AAk?$AAe?$AAr?$AAn?$AAe?$AAl?$AA3?$AA2?$AA?4?$AAd?$AAl?$AAl@ 0000000180007238     MSVCRT:thread_safe_statics.obj
 0002:00002258       ??_C@_0BJ@JEBJOJFJ@SleepConditionVariableCS@ 0000000180007258     MSVCRT:thread_safe_statics.obj
 0002:00002278       ??_C@_0BJ@PGPPEPCC@WakeAllConditionVariable@ 0000000180007278     MSVCRT:thread_safe_statics.obj
 0002:00002298       _pDefaultRawDllMain        0000000180007298     MSVCRT:dll_dllmain.obj
 0002:00002298       _pRawDllMain               0000000180007298     MSVCRT:dll_dllmain.obj
 0002:000022a0       __xmm@ffffffffffffffffffffffffffffffff 00000001800072a0     MSVCRT:utility.obj
 0002:000022b0       _load_config_used          00000001800072b0     MSVCRT:loadcfg.obj
 0002:00002480       _tls_used                  0000000180007480     MSVCRT:tlssup.obj
 0002:000024a8       __volatile_metadata        00000001800074a8     <linker-defined>
 0002:00002878       __rtc_iaa                  0000000180007878     MSVCRT:initsect.obj
 0002:00002880       __rtc_izz                  0000000180007880     MSVCRT:initsect.obj
 0002:00002888       __rtc_taa                  0000000180007888     MSVCRT:initsect.obj
 0002:00002890       __rtc_tzz                  0000000180007890     MSVCRT:initsect.obj
 0002:00002898       _tls_start                 0000000180007898     MSVCRT:tlssup.obj
 0002:0000289c       _Init_thread_epoch         000000018000789c     MSVCRT:thread_safe_statics.obj
 0002:000028a0       _tls_end                   00000001800078a0     MSVCRT:tlssup.obj
 0002:00002fa0       __IMPORT_DESCRIPTOR_KERNEL32 0000000180007fa0     kernel32:KERNEL32.dll
 0002:00002fb4       __IMPORT_DESCRIPTOR_VCRUNTIME140 0000000180007fb4     vcruntime:VCRUNTIME140.dll
 0002:00002fc8       __IMPORT_DESCRIPTOR_api-ms-win-crt-heap-l1-1-0 0000000180007fc8     ucrt:api-ms-win-crt-heap-l1-1-0.dll
 0002:00002fdc       __IMPORT_DESCRIPTOR_api-ms-win-crt-runtime-l1-1-0 0000000180007fdc     ucrt:api-ms-win-crt-runtime-l1-1-0.dll
 0002:00002ff0       __IMPORT_DESCRIPTOR_api-ms-win-crt-convert-l1-1-0 0000000180007ff0     ucrt:api-ms-win-crt-convert-l1-1-0.dll
 0002:00003004       __IMPORT_DESCRIPTOR_api-ms-win-crt-stdio-l1-1-0 0000000180008004     ucrt:api-ms-win-crt-stdio-l1-1-0.dll
 0002:00003018       __IMPORT_DESCRIPTOR_api-ms-win-crt-string-l1-1-0 0000000180008018     ucrt:api-ms-win-crt-string-l1-1-0.dll
 0002:0000302c       __NULL_IMPORT_DESCRIPTOR   000000018000802c     kernel32:KERNEL32.dll
 0003:00000000       jvmti_phase_to_check       0000000180009000     libsystemclssearch_agent.obj
 0003:00000034       _Init_global_epoch         0000000180009034     MSVCRT:thread_safe_statics.obj
 0003:00000040       __security_cookie          0000000180009040     MSVCRT:gs_cookie.obj
 0003:00000048       __security_cookie_complement 0000000180009048     MSVCRT:gs_cookie.obj
 0003:00000050       __scrt_native_dllmain_reason 0000000180009050     MSVCRT:utility.obj
 0003:00000058       __isa_available            0000000180009058     MSVCRT:cpu_disp.obj
 0003:0000005c       __isa_enabled              000000018000905c     MSVCRT:cpu_disp.obj
 0003:00000060       __memset_fast_string_threshold 0000000180009060     MSVCRT:cpu_disp.obj
 0003:00000068       __memset_nt_threshold      0000000180009068     MSVCRT:cpu_disp.obj
 0003:00000070       __scrt_ucrt_dll_is_in_use  0000000180009070     MSVCRT:ucrt_stubs.obj
 0003:00000080       g_wrongHeapCallbacks       0000000180009080     libsystemclssearch_agent.obj
 0003:00000100       g_szTagInfo                0000000180009100     libsystemclssearch_agent.obj
 0003:00002040       g_tagFlags                 000000018000b040     libsystemclssearch_agent.obj
 0003:00002428       g_refsToVerifyCnt          000000018000b428     libsystemclssearch_agent.obj
 0003:0000242c       g_fakeUserData             000000018000b42c     libsystemclssearch_agent.obj
 0003:00002430       g_tagVisitCount            000000018000b430     libsystemclssearch_agent.obj
 0003:000033d0       g_refsToVerify             000000018000c3d0     libsystemclssearch_agent.obj
 0003:0001aad0       g_userDataError            0000000180023ad0     libsystemclssearch_agent.obj
 0003:0001aad4       use_segment2               0000000180023ad4     libsystemclssearch_agent.obj
 0003:0001c3e8       ?_OptionsStorage@?1??__local_stdio_printf_options@@9@4_KA 00000001800253e8     libsystemclssearch_agent.obj
 0003:0001c9a8       _tls_index                 00000001800259a8     MSVCRT:tlssup.obj
 0003:0001c9b0       __scrt_current_native_startup_state 00000001800259b0     MSVCRT:utility.obj
 0003:0001c9b8       __scrt_native_startup_lock 00000001800259b8     MSVCRT:utility.obj
 0003:0001c9f8       __scrt_debugger_hook_flag  00000001800259f8     MSVCRT:utility_desktop.obj
 0003:0001ca00       ?__type_info_root_node@@3U__type_info_node@@A 0000000180025a00     MSVCRT:tncleanup.obj
 0003:0001ca10       ?_OptionsStorage@?1??__local_stdio_scanf_options@@9@4_KA 0000000180025a10     MSVCRT:default_local_stdio_options.obj
 0003:0001ca18       __favor                    0000000180025a18     MSVCRT:cpu_disp.obj
 0003:0001ca20       __dyn_tls_init_callback    0000000180025a20     <common>

 entry point at        0001:00002f70

 Static symbols

 0000:fffd8000       .debug$S                   0000000180000000     systemclssearch_agent.exp
 0000:fffd8000       .debug$S                   0000000180000000     vcruntime:VCRUNTIME140.dll
 0000:fffd8000       .debug$S                   0000000180000000     vcruntime:VCRUNTIME140.dll
 0000:fffd8000       .debug$S                   0000000180000000     vcruntime:VCRUNTIME140.dll
 0000:fffd8000       .debug$S                   0000000180000000     vcruntime:VCRUNTIME140.dll
 0000:fffd8000       .debug$S                   0000000180000000     vcruntime:VCRUNTIME140.dll
 0000:fffd8000       .debug$S                   0000000180000000     vcruntime:VCRUNTIME140.dll
 0000:fffd8000       .debug$S                   0000000180000000     vcruntime:VCRUNTIME140.dll
 0000:fffd8000       .debug$S                   0000000180000000     ucrt:api-ms-win-crt-convert-l1-1-0.dll
 0000:fffd8000       .debug$S                   0000000180000000     ucrt:api-ms-win-crt-heap-l1-1-0.dll
 0000:fffd8000       .debug$S                   0000000180000000     ucrt:api-ms-win-crt-heap-l1-1-0.dll
 0000:fffd8000       .debug$S                   0000000180000000     ucrt:api-ms-win-crt-heap-l1-1-0.dll
 0000:fffd8000       .debug$S                   0000000180000000     ucrt:api-ms-win-crt-heap-l1-1-0.dll
 0000:fffd8000       .debug$S                   0000000180000000     ucrt:api-ms-win-crt-runtime-l1-1-0.dll
 0000:fffd8000       .debug$S                   0000000180000000     ucrt:api-ms-win-crt-runtime-l1-1-0.dll
 0000:fffd8000       .debug$S                   0000000180000000     ucrt:api-ms-win-crt-runtime-l1-1-0.dll
 0000:fffd8000       .debug$S                   0000000180000000     ucrt:api-ms-win-crt-runtime-l1-1-0.dll
 0000:fffd8000       .debug$S                   0000000180000000     ucrt:api-ms-win-crt-runtime-l1-1-0.dll
 0000:fffd8000       .debug$S                   0000000180000000     ucrt:api-ms-win-crt-runtime-l1-1-0.dll
 0000:fffd8000       .debug$S                   0000000180000000     ucrt:api-ms-win-crt-runtime-l1-1-0.dll
 0000:fffd8000       .debug$S                   0000000180000000     ucrt:api-ms-win-crt-runtime-l1-1-0.dll
 0000:fffd8000       .debug$S                   0000000180000000     ucrt:api-ms-win-crt-runtime-l1-1-0.dll
 0000:fffd8000       .debug$S                   0000000180000000     ucrt:api-ms-win-crt-runtime-l1-1-0.dll
 0000:fffd8000       .debug$S                   0000000180000000     ucrt:api-ms-win-crt-runtime-l1-1-0.dll
 0000:fffd8000       .debug$S                   0000000180000000     ucrt:api-ms-win-crt-runtime-l1-1-0.dll
 0000:fffd8000       .debug$S                   0000000180000000     ucrt:api-ms-win-crt-runtime-l1-1-0.dll
 0000:fffd8000       .debug$S                   0000000180000000     ucrt:api-ms-win-crt-runtime-l1-1-0.dll
 0000:fffd8000       .debug$S                   0000000180000000     ucrt:api-ms-win-crt-runtime-l1-1-0.dll
 0000:fffd8000       .debug$S                   0000000180000000     ucrt:api-ms-win-crt-runtime-l1-1-0.dll
 0000:fffd8000       .debug$S                   0000000180000000     ucrt:api-ms-win-crt-stdio-l1-1-0.dll
 0000:fffd8000       .debug$S                   0000000180000000     ucrt:api-ms-win-crt-stdio-l1-1-0.dll
 0000:fffd8000       .debug$S                   0000000180000000     ucrt:api-ms-win-crt-stdio-l1-1-0.dll
 0000:fffd8000       .debug$S                   0000000180000000     ucrt:api-ms-win-crt-stdio-l1-1-0.dll
 0000:fffd8000       .debug$S                   0000000180000000     ucrt:api-ms-win-crt-stdio-l1-1-0.dll
 0000:fffd8000       .debug$S                   0000000180000000     ucrt:api-ms-win-crt-stdio-l1-1-0.dll
 0000:fffd8000       .debug$S                   0000000180000000     ucrt:api-ms-win-crt-stdio-l1-1-0.dll
 0000:fffd8000       .debug$S                   0000000180000000     ucrt:api-ms-win-crt-stdio-l1-1-0.dll
 0000:fffd8000       .debug$S                   0000000180000000     ucrt:api-ms-win-crt-stdio-l1-1-0.dll
 0000:fffd8000       .debug$S                   0000000180000000     ucrt:api-ms-win-crt-stdio-l1-1-0.dll
 0000:fffd8000       .debug$S                   0000000180000000     ucrt:api-ms-win-crt-string-l1-1-0.dll
 0000:fffd8000       .debug$S                   0000000180000000     ucrt:api-ms-win-crt-string-l1-1-0.dll
 0000:fffd8000       .debug$S                   0000000180000000     ucrt:api-ms-win-crt-string-l1-1-0.dll
 0000:fffd8000       .debug$S                   0000000180000000     ucrt:api-ms-win-crt-string-l1-1-0.dll
 0000:fffd8000       .debug$S                   0000000180000000     ucrt:api-ms-win-crt-string-l1-1-0.dll
 0000:fffd8000       .debug$S                   0000000180000000     ucrt:api-ms-win-crt-string-l1-1-0.dll
 0000:fffd8000       .debug$S                   0000000180000000     ucrt:api-ms-win-crt-string-l1-1-0.dll
 0000:fffd8000       .debug$S                   0000000180000000     ucrt:api-ms-win-crt-string-l1-1-0.dll
 0000:fffd8000       .debug$S                   0000000180000000     kernel32:KERNEL32.dll
 0000:fffd8000       .debug$S                   0000000180000000     kernel32:KERNEL32.dll
 0000:fffd8000       .debug$S                   0000000180000000     kernel32:KERNEL32.dll
 0000:fffd8000       .debug$S                   0000000180000000     kernel32:KERNEL32.dll
 0000:fffd8000       .debug$S                   0000000180000000     kernel32:KERNEL32.dll
 0000:fffd8000       .debug$S                   0000000180000000     kernel32:KERNEL32.dll
 0000:fffd8000       .debug$S                   0000000180000000     kernel32:KERNEL32.dll
 0000:fffd8000       .debug$S                   0000000180000000     kernel32:KERNEL32.dll
 0000:fffd8000       .debug$S                   0000000180000000     kernel32:KERNEL32.dll
 0000:fffd8000       .debug$S                   0000000180000000     kernel32:KERNEL32.dll
 0000:fffd8000       .debug$S                   0000000180000000     kernel32:KERNEL32.dll
 0000:fffd8000       .debug$S                   0000000180000000     kernel32:KERNEL32.dll
 0000:fffd8000       .debug$S                   0000000180000000     kernel32:KERNEL32.dll
 0000:fffd8000       .debug$S                   0000000180000000     kernel32:KERNEL32.dll
 0000:fffd8000       .debug$S                   0000000180000000     kernel32:KERNEL32.dll
 0000:fffd8000       .debug$S                   0000000180000000     kernel32:KERNEL32.dll
 0000:fffd8000       .debug$S                   0000000180000000     kernel32:KERNEL32.dll
 0000:fffd8000       .debug$S                   0000000180000000     kernel32:KERNEL32.dll
 0000:fffd8000       .debug$S                   0000000180000000     kernel32:KERNEL32.dll
 0000:fffd8000       .debug$S                   0000000180000000     kernel32:KERNEL32.dll
 0000:fffd8000       .debug$S                   0000000180000000     kernel32:KERNEL32.dll
 0000:fffd8000       .debug$S                   0000000180000000     kernel32:KERNEL32.dll
 0000:fffd8000       .debug$S                   0000000180000000     kernel32:KERNEL32.dll
 0000:fffd8000       .debug$S                   0000000180000000     kernel32:KERNEL32.dll
 0000:fffd8000       .debug$S                   0000000180000000     kernel32:KERNEL32.dll
 0000:fffd8000       .debug$S                   0000000180000000     kernel32:KERNEL32.dll
 0000:fffd8000       .debug$S                   0000000180000000     kernel32:KERNEL32.dll
 0000:fffd8000       .debug$S                   0000000180000000     kernel32:KERNEL32.dll
 0001:00001084       addRefToVerify             0000000180002084 f   libsystemclssearch_agent.obj
 0001:000010f0       addSegment                 00000001800020f0 f   libsystemclssearch_agent.obj
 0001:000011dc       agentThreadWrapper         00000001800021dc f   libsystemclssearch_agent.obj
 0001:00001528       checkLivePhaseForIllegalArgs 0000000180002528 f   libsystemclssearch_agent.obj
 0001:00001634       check_option               0000000180002634 f   libsystemclssearch_agent.obj
 0001:0000187c       file_basename              000000018000287c f   libsystemclssearch_agent.obj
 0001:00002450       startAgentThreadWrapper    0000000180003450 f   libsystemclssearch_agent.obj
 0001:00002790       syncDebuggeeStatus         0000000180003790 f   libsystemclssearch_agent.obj
 0001:00002a30       capture_previous_context   0000000180003a30 f   MSVCRT:gs_report.obj
 0001:00002aa4       ?__scrt_initialize_thread_safe_statics@@YAHXZ 0000000180003aa4 f   MSVCRT:thread_safe_statics.obj
 0001:00002b74       ?__scrt_uninitialize_thread_safe_statics@@YAXXZ 0000000180003b74 f   MSVCRT:thread_safe_statics.obj
 0001:00002c20       $$000000                   0000000180003c20     MSVCRT:amdsecgs.obj
 0001:00002c50       ?dllmain_crt_dispatch@@YAHQEAUHINSTANCE__@@KQEAX@Z 0000000180003c50 f   MSVCRT:dll_dllmain.obj
 0001:00002ca0       ?dllmain_crt_process_attach@@YAHQEAUHINSTANCE__@@QEAX@Z 0000000180003ca0 f   MSVCRT:dll_dllmain.obj
 0001:00002db8       ?dllmain_crt_process_detach@@YAH_N@Z 0000000180003db8 f   MSVCRT:dll_dllmain.obj
 0001:00002e3c       ?dllmain_dispatch@@YAHQEAUHINSTANCE__@@KQEAX@Z 0000000180003e3c f   MSVCRT:dll_dllmain.obj
 0001:00003850       $$000000                   0000000180004850     MSVCRT:guard_dispatch.obj
 0001:00003870       $$000000                   0000000180004870     MSVCRT:guard_xfg_dispatch.obj
 0001:00003886       ?fin$0@?0??dllmain_crt_process_attach@@YAHQEAUHINSTANCE__@@QEAX@Z@4HA 0000000180004886 f   MSVCRT:dll_dllmain.obj
 0001:0000389d       ?fin$0@?0??dllmain_crt_process_detach@@YAH_N@Z@4HA 000000018000489d f   MSVCRT:dll_dllmain.obj
 0001:000038b6       ?fin$1@?0??dllmain_crt_process_detach@@YAH_N@Z@4HA 00000001800048b6 f   MSVCRT:dll_dllmain.obj
 0001:000038ca       ?filt$0@?0??dllmain_dispatch@@YAHQEAUHINSTANCE__@@KQEAX@Z@4HA 00000001800048ca f   MSVCRT:dll_dllmain.obj
 0001:00003900       __scrt_is_nonwritable_in_current_image$filt$0 0000000180004900 f   MSVCRT:utility.obj
 0002:00000218       ?__scrt_initialize_tss_var@@3P6AHXZEA 0000000180005218     MSVCRT:thread_safe_statics.obj
 0002:00000340       ?opcLengths@@3QBEB         0000000180005340     libsystemclssearch_agent.obj
 0002:00000410       illegal_segments           0000000180005410     libsystemclssearch_agent.obj
 0002:000021d8       GS_ExceptionPointers       00000001800071d8     MSVCRT:gs_report.obj
 0002:000028a8       $unwind$fprintf            00000001800078a8     libsystemclssearch_agent.obj
 0002:000028b4       $unwind$printf             00000001800078b4     libsystemclssearch_agent.obj
 0002:000028c0       $unwind$?NewObject@JNIEnv_@@QEAAPEAV_jobject@@PEAV_jclass@@PEAU_jmethodID@@ZZ 00000001800078c0     libsystemclssearch_agent.obj
 0002:000028c0       $unwind$nsk_lcomplain      00000001800078c0     libsystemclssearch_agent.obj
 0002:000028c0       $unwind$nsk_ldisplay       00000001800078c0     libsystemclssearch_agent.obj
 0002:000028c8       $unwind$nsk_lvdisplay      00000001800078c8     libsystemclssearch_agent.obj
 0002:000028c8       $unwind$_RTC_Initialize    00000001800078c8     MSVCRT:initsect.obj
 0002:000028c8       $unwind$_RTC_Terminate     00000001800078c8     MSVCRT:initsect.obj
 0002:000028c8       $unwind$?__scrt_initialize_thread_safe_statics@@YAHXZ 00000001800078c8     MSVCRT:thread_safe_statics.obj
 0002:000028d4       $unwind$nsk_complain       00000001800078d4     libsystemclssearch_agent.obj
 0002:000028d4       $unwind$nsk_printf         00000001800078d4     libsystemclssearch_agent.obj
 0002:000028dc       $unwind$nsk_lvcomplain     00000001800078dc     libsystemclssearch_agent.obj
 0002:000028f4       $unwind$nsk_ltrace         00000001800078f4     libsystemclssearch_agent.obj
 0002:000028f4       $unwind$__report_gsfailure 00000001800078f4     MSVCRT:gs_report.obj
 0002:000028fc       $unwind$callbackVMInit     00000001800078fc     libsystemclssearch_agent.obj
 0002:000028fc       $unwind$nsk_lvtrace        00000001800078fc     libsystemclssearch_agent.obj
 0002:000028fc       $unwind$__raise_securityfailure 00000001800078fc     MSVCRT:gs_report.obj
 0002:000028fc       $unwind$__scrt_initialize_crt 00000001800078fc     MSVCRT:utility.obj
 0002:000028fc       $unwind$__scrt_initialize_onexit_tables 00000001800078fc     MSVCRT:utility.obj
 0002:000028fc       $unwind$__scrt_release_startup_lock 00000001800078fc     MSVCRT:utility.obj
 0002:000028fc       $unwind$__scrt_uninitialize_crt 00000001800078fc     MSVCRT:utility.obj
 0002:000028fc       $unwind$_onexit            00000001800078fc     MSVCRT:utility.obj
 0002:00002904       $unwind$nsk_lverify        0000000180007904     libsystemclssearch_agent.obj
 0002:00002914       $unwind$nsk_vprintf        0000000180007914     libsystemclssearch_agent.obj
 0002:00002924       $unwind$?nsk_jni_lverify@@YAHHPEAUJNIEnv_@@HQEBDH1ZZ 0000000180007924     libsystemclssearch_agent.obj
 0002:00002938       $unwind$?nsk_jni_check_exception@@YAHPEAUJNIEnv_@@QEBDH@Z 0000000180007938     libsystemclssearch_agent.obj
 0002:00002954       $unwind$nsk_jvmti_parseOptions 0000000180007954     libsystemclssearch_agent.obj
 0002:00002970       $unwind$nsk_jvmti_createJVMTIEnv 0000000180007970     libsystemclssearch_agent.obj
 0002:00002984       $unwind$Java_nsk_jvmti_unit_FollowReferences_FollowRefObjects_resetTags 0000000180007984     libsystemclssearch_agent.obj
 0002:00002984       $unwind$addRefToVerify     0000000180007984     libsystemclssearch_agent.obj
 0002:00002984       $unwind$nsk_jvmti_resetAgentData 0000000180007984     libsystemclssearch_agent.obj
 0002:00002984       $unwind$nsk_jvmti_setFailStatus 0000000180007984     libsystemclssearch_agent.obj
 0002:00002984       $unwind$__scrt_initialize_default_local_stdio_options 0000000180007984     MSVCRT:default_local_stdio_options.obj
 0002:00002984       $unwind$?dllmain_crt_dispatch@@YAHQEAUHINSTANCE__@@KQEAX@Z 0000000180007984     MSVCRT:dll_dllmain.obj
 0002:00002984       $unwind$DllMain            0000000180007984     MSVCRT:dll_dllmain_stub.obj
 0002:00002984       $unwind$__GSHandlerCheck   0000000180007984     MSVCRT:gshandler.obj
 0002:00002984       $unwind$?__scrt_uninitialize_thread_safe_statics@@YAXXZ 0000000180007984     MSVCRT:thread_safe_statics.obj
 0002:00002984       $unwind$__scrt_acquire_startup_lock 0000000180007984     MSVCRT:utility.obj
 0002:00002984       $unwind$__scrt_dllmain_after_initialize_c 0000000180007984     MSVCRT:utility.obj
 0002:00002984       $unwind$__scrt_dllmain_before_initialize_c 0000000180007984     MSVCRT:utility.obj
 0002:00002984       $unwind$__scrt_dllmain_crt_thread_attach 0000000180007984     MSVCRT:utility.obj
 0002:00002984       $unwind$__scrt_dllmain_crt_thread_detach 0000000180007984     MSVCRT:utility.obj
 0002:00002984       $unwind$__scrt_dllmain_uninitialize_c 0000000180007984     MSVCRT:utility.obj
 0002:00002984       $unwind$__scrt_dllmain_uninitialize_critical 0000000180007984     MSVCRT:utility.obj
 0002:00002984       $unwind$atexit             0000000180007984     MSVCRT:utility.obj
 0002:0000298c       $unwind$nsk_jvmti_enableEvents 000000018000798c     libsystemclssearch_agent.obj
 0002:000029a4       $unwind$check_option       00000001800079a4     libsystemclssearch_agent.obj
 0002:000029a4       $unwind$nsk_jvmti_findOptionStringValue 00000001800079a4     libsystemclssearch_agent.obj
 0002:000029a4       $unwind$nsk_jvmti_findOptionValue 00000001800079a4     libsystemclssearch_agent.obj
 0002:000029a4       $unwind$_DllMainCRTStartup 00000001800079a4     MSVCRT:dll_dllmain.obj
 0002:000029b4       $unwind$nsk_jvmti_lverify  00000001800079b4     libsystemclssearch_agent.obj
 0002:000029c8       $unwind$exitOnError        00000001800079c8     libsystemclssearch_agent.obj
 0002:000029d8       $unwind$Java_nsk_share_jvmti_ArgumentHandler_getAgentOptionsString 00000001800079d8     libsystemclssearch_agent.obj
 0002:000029ec       $unwind$Java_nsk_jvmti_unit_FollowReferences_FollowRefObjects_getTag 00000001800079ec     libsystemclssearch_agent.obj
 0002:000029ec       $unwind$Java_nsk_share_jvmti_DebugeeClass_checkStatus 00000001800079ec     libsystemclssearch_agent.obj
 0002:000029ec       $unwind$agentThreadWrapper 00000001800079ec     libsystemclssearch_agent.obj
 0002:000029fc       $unwind$startAgentThreadWrapper 00000001800079fc     libsystemclssearch_agent.obj
 0002:00002a18       $unwind$syncDebuggeeStatus 0000000180007a18     libsystemclssearch_agent.obj
 0002:00002a18       $unwind$__scrt_dllmain_exception_filter 0000000180007a18     MSVCRT:utility.obj
 0002:00002a2c       $unwind$Java_nsk_share_jvmti_DebugeeClass_resetAgentData 0000000180007a2c     libsystemclssearch_agent.obj
 0002:00002a34       $unwind$MA_checkStatus     0000000180007a34     libsystemclssearch_agent.obj
 0002:00002a48       $unwind$Java_nsk_jvmti_unit_FollowReferences_FollowRefObjects_setTag 0000000180007a48     libsystemclssearch_agent.obj
 0002:00002a60       $unwind$Java_nsk_jvmti_unit_FollowReferences_FollowRefObjects_addRefToVerify 0000000180007a60     libsystemclssearch_agent.obj
 0002:00002a7c       $unwind$Agent_Initialize   0000000180007a7c     libsystemclssearch_agent.obj
 0002:00002a9c       $unwind$addSegment         0000000180007a9c     libsystemclssearch_agent.obj
 0002:00002ab4       $unwind$checkLivePhaseForIllegalArgs 0000000180007ab4     libsystemclssearch_agent.obj
 0002:00002acc       $unwind$callbackVMDeath    0000000180007acc     libsystemclssearch_agent.obj
 0002:00002ae0       $unwind$capture_previous_context 0000000180007ae0     MSVCRT:gs_report.obj
 0002:00002aec       $unwind$__GSHandlerCheckCommon 0000000180007aec     MSVCRT:gshandler.obj
 0002:00002af8       $xdatasym                  0000000180007af8     MSVCRT:amdsecgs.obj
 0002:00002afc       $unwind$?dllmain_crt_process_attach@@YAHQEAUHINSTANCE__@@QEAX@Z 0000000180007afc     MSVCRT:dll_dllmain.obj
 0002:00002b38       $unwind$?fin$0@?0??dllmain_crt_process_attach@@YAHQEAUHINSTANCE__@@QEAX@Z@4HA 0000000180007b38     MSVCRT:dll_dllmain.obj
 0002:00002b38       $unwind$?fin$0@?0??dllmain_crt_process_detach@@YAH_N@Z@4HA 0000000180007b38     MSVCRT:dll_dllmain.obj
 0002:00002b38       $unwind$?fin$1@?0??dllmain_crt_process_detach@@YAH_N@Z@4HA 0000000180007b38     MSVCRT:dll_dllmain.obj
 0002:00002b40       $unwind$?dllmain_crt_process_detach@@YAH_N@Z 0000000180007b40     MSVCRT:dll_dllmain.obj
 0002:00002b94       $unwind$?dllmain_dispatch@@YAHQEAUHINSTANCE__@@KQEAX@Z 0000000180007b94     MSVCRT:dll_dllmain.obj
 0002:00002bbc       $unwind$?filt$0@?0??dllmain_dispatch@@YAHQEAUHINSTANCE__@@KQEAX@Z@4HA 0000000180007bbc     MSVCRT:dll_dllmain.obj
 0002:00002bc4       $unwind$__scrt_is_nonwritable_in_current_image 0000000180007bc4     MSVCRT:utility.obj
 0002:00002be4       $unwind$__scrt_is_nonwritable_in_current_image$filt$0 0000000180007be4     MSVCRT:utility.obj
 0002:00002bec       $unwind$__scrt_fastfail    0000000180007bec     MSVCRT:utility_desktop.obj
 0002:00002bfc       $unwind$__security_init_cookie 0000000180007bfc     MSVCRT:gs_support.obj
 0002:00002c08       $unwind$__isa_available_init 0000000180007c08     MSVCRT:cpu_disp.obj
 0002:00002c18       $xdatasym                  0000000180007c18     MSVCRT:guard_dispatch.obj
 0002:00002c20       $xdatasym                  0000000180007c20     MSVCRT:guard_xfg_dispatch.obj
 0002:00002c30       .edata                     0000000180007c30     systemclssearch_agent.exp
 0002:00002c58       rgpv                       0000000180007c58     systemclssearch_agent.exp
 0002:00002c90       rgszName                   0000000180007c90     systemclssearch_agent.exp
 0002:00002cc8       rgwOrd                     0000000180007cc8     systemclssearch_agent.exp
 0002:00002ce4       szName                     0000000180007ce4     systemclssearch_agent.exp
 0002:00002cfe       $N00001                    0000000180007cfe     systemclssearch_agent.exp
 0002:00002d0d       $N00002                    0000000180007d0d     systemclssearch_agent.exp
 0002:00002d1a       $N00003                    0000000180007d1a     systemclssearch_agent.exp
 0002:00002d5f       $N00004                    0000000180007d5f     systemclssearch_agent.exp
 0002:00002d9c       $N00005                    0000000180007d9c     systemclssearch_agent.exp
 0002:00002de4       $N00006                    0000000180007de4     systemclssearch_agent.exp
 0002:00002e24       $N00007                    0000000180007e24     systemclssearch_agent.exp
 0002:00002e61       $N00008                    0000000180007e61     systemclssearch_agent.exp
 0002:00002e9c       $N00009                    0000000180007e9c     systemclssearch_agent.exp
 0002:00002eca       $N00010                    0000000180007eca     systemclssearch_agent.exp
 0002:00002efb       $N00011                    0000000180007efb     systemclssearch_agent.exp
 0002:00002f2a       $N00012                    0000000180007f2a     systemclssearch_agent.exp
 0002:00002f59       $N00013                    0000000180007f59     systemclssearch_agent.exp
 0002:00002f8e       $N00014                    0000000180007f8e     systemclssearch_agent.exp
 0002:000033f2       .idata$6                   00000001800083f2     kernel32:KERNEL32.dll
 0002:00003456       .idata$6                   0000000180008456     vcruntime:VCRUNTIME140.dll
 0002:000035e8       .idata$6                   00000001800085e8     ucrt:api-ms-win-crt-heap-l1-1-0.dll
 0002:00003608       .idata$6                   0000000180008608     ucrt:api-ms-win-crt-runtime-l1-1-0.dll
 0002:0000362a       .idata$6                   000000018000862a     ucrt:api-ms-win-crt-convert-l1-1-0.dll
 0002:0000364c       .idata$6                   000000018000864c     ucrt:api-ms-win-crt-stdio-l1-1-0.dll
 0002:0000366c       .idata$6                   000000018000866c     ucrt:api-ms-win-crt-string-l1-1-0.dll
 0003:00000004       ?callBytes@@3PAEA          0000000180009004     libsystemclssearch_agent.obj
 0003:00000008       ?codeAttributeName@@3PEBDEB 0000000180009008     libsystemclssearch_agent.obj
 0003:00000010       ?lineNumberAttributeName@@3PEBDEB 0000000180009010     libsystemclssearch_agent.obj
 0003:00000018       ?localVarAttributeName@@3PEBDEB 0000000180009018     libsystemclssearch_agent.obj
 0003:00000020       ?localVarTypeAttributeName@@3PEBDEB 0000000180009020     libsystemclssearch_agent.obj
 0003:00000028       ?stackMapAttributeName@@3PEBDEB 0000000180009028     libsystemclssearch_agent.obj
 0003:00000030       ?allocBytes@@3PAEA         0000000180009030     libsystemclssearch_agent.obj
 0003:0001aad8       nsk_context                0000000180023ad8     libsystemclssearch_agent.obj
 0003:0001aae4       redefineAttempted          0000000180023ae4     libsystemclssearch_agent.obj
 0003:0001aae8       redefineSucceed            0000000180023ae8     libsystemclssearch_agent.obj
 0003:0001aaec       agentFailed                0000000180023aec     libsystemclssearch_agent.obj
 0003:0001aaf0       context                    0000000180023af0     libsystemclssearch_agent.obj
 0003:0001aba8       agentThread                0000000180023ba8     libsystemclssearch_agent.obj
 0003:0001abb0       agentThreadProc            0000000180023bb0     libsystemclssearch_agent.obj
 0003:0001abb8       agentThreadArg             0000000180023bb8     libsystemclssearch_agent.obj
 0003:0001abc0       agent_data                 0000000180023bc0     libsystemclssearch_agent.obj
 0003:0001abd0       jvmti_env                  0000000180023bd0     libsystemclssearch_agent.obj
 0003:0001abd8       jvm                        0000000180023bd8     libsystemclssearch_agent.obj
 0003:0001abe0       jni_env                    0000000180023be0     libsystemclssearch_agent.obj
 0003:0001abe8       currentAgentStatus         0000000180023be8     libsystemclssearch_agent.obj
 0003:0001abec       ?codeAttributeIndex@@3GA   0000000180023bec     libsystemclssearch_agent.obj
 0003:0001abf0       checkStatus_func           0000000180023bf0     libsystemclssearch_agent.obj
 0003:0001abf8       ?lineNumberAttributeIndex@@3GA 0000000180023bf8     libsystemclssearch_agent.obj
 0003:0001abfc       ?localVarAttributeIndex@@3GA 0000000180023bfc     libsystemclssearch_agent.obj
 0003:0001ac00       ?localVarTypeAttributeIndex@@3GA 0000000180023c00     libsystemclssearch_agent.obj
 0003:0001ac04       ?stackMapAttributeIndex@@3GA 0000000180023c04     libsystemclssearch_agent.obj
 0003:0001ac08       ?stackFrameOffset@@3GA     0000000180023c08     libsystemclssearch_agent.obj
 0003:0001ac0c       ?mode@@3HA                 0000000180023c0c     libsystemclssearch_agent.obj
 0003:0001ac10       ?orig@@3PEBEEB             0000000180023c10     libsystemclssearch_agent.obj
 0003:0001ac18       ?gen@@3PEAEEA              0000000180023c18     libsystemclssearch_agent.obj
 0003:0001ac20       ?inputPos@@3PEAEEA         0000000180023c20     libsystemclssearch_agent.obj
 0003:0001ac28       ?endPos@@3PEBEEB           0000000180023c28     libsystemclssearch_agent.obj
 0003:0001ac30       ?genPos@@3PEAEEA           0000000180023c30     libsystemclssearch_agent.obj
 0003:0001ac38       ?markPos@@3PEAEEA          0000000180023c38     libsystemclssearch_agent.obj
 0003:0001ac40       ?constantPool@@3PEAPEADEA  0000000180023c40     libsystemclssearch_agent.obj
 0003:0001ac48       ?constantPoolSize@@3GA     0000000180023c48     libsystemclssearch_agent.obj
 0003:0001ac4c       ?constantPoolCount@@3GA    0000000180023c4c     libsystemclssearch_agent.obj
 0003:0001ac50       ?zeroBytes@@3PAEA          0000000180023c50     libsystemclssearch_agent.obj
 0003:0001ac54       ?codeLength@@3IA           0000000180023c54     libsystemclssearch_agent.obj
 0003:0001ac58       ?map@@3PEAIEA              0000000180023c58     libsystemclssearch_agent.obj
 0003:0001ac60       ?widening@@3PEACEA         0000000180023c60     libsystemclssearch_agent.obj
 0003:0001ac68       timeout                    0000000180023c68     libsystemclssearch_agent.obj
 0003:0001ac70       segment1                   0000000180023c70     libsystemclssearch_agent.obj
 0003:0001b830       segment2                   0000000180024830     libsystemclssearch_agent.obj
 0003:0001c3f0       GS_ExceptionRecord         00000001800253f0     MSVCRT:gs_report.obj
 0003:0001c490       GS_ContextRecord           0000000180025490     MSVCRT:gs_report.obj
 0003:0001c960       ?g_tss_cv@@3U_RTL_CONDITION_VARIABLE@@A 0000000180025960     MSVCRT:thread_safe_statics.obj
 0003:0001c968       ?g_tss_event@@3PEAXEA      0000000180025968     MSVCRT:thread_safe_statics.obj
 0003:0001c970       ?g_tss_mutex@@3U_RTL_CRITICAL_SECTION@@A 0000000180025970     MSVCRT:thread_safe_statics.obj
 0003:0001c998       ?g_sleep_condition_variable_cs@@3P6AHPEAU_RTL_CONDITION_VARIABLE@@PEAU_RTL_CRITICAL_SECTION@@K@ZEA 0000000180025998     MSVCRT:thread_safe_statics.obj
 0003:0001c9a0       ?g_wake_all_condition_variable@@3P6AXPEAU_RTL_CONDITION_VARIABLE@@@ZEA 00000001800259a0     MSVCRT:thread_safe_statics.obj
 0003:0001c9ac       ?__proc_attached@@3HA      00000001800259ac     MSVCRT:dll_dllmain.obj
 0003:0001c9c0       ?is_initialized_as_dll@@3_NA 00000001800259c0     MSVCRT:utility.obj
 0003:0001c9c1       ?module_local_atexit_table_initialized@@3_NA 00000001800259c1     MSVCRT:utility.obj
 0003:0001c9c8       ?module_local_atexit_table@@3U_onexit_table_t@@A 00000001800259c8     MSVCRT:utility.obj
 0003:0001c9e0       ?module_local_at_quick_exit_table@@3U_onexit_table_t@@A 00000001800259e0     MSVCRT:utility.obj
